:020000041000EA
:1000000000B5324B212058609868022188439860DF
:10001000D860186158612E4B002199600221596106
:100020000121F02299502B49196001219960352056
:1000300000F044F80222904214D00621196600F024
:1000400034F8196E01211966002018661A6600F04E
:100050002CF8196E196E196E052000F02FF8012189
:100060000842F9D1002199601B49196000215960AB
:100070001A491B48016001219960EB211966A021F2
:10008000196600F012F800219960164914480160C1
:100090000121996001BC002800D000471248134993
:1000A000086003C880F30888084703B5996A0420EC
:1000B0000142FBD001200142F8D103BD02B5186610
:1000C0001866FFF7F2FF186E186E02BD00000240BE
:1000D000000000180000070000035F00212200005C
:1000E000F4000018222000A00001001008ED00E03C
:1000F00000000000000000000000000074B24E7A12
:1001000000200420F7010010C3010010C5010010F9
:10011000C1010010C1010010C1010010C101001097
:10012000C1010010C1010010C1010010C701001081
:10013000C1010010C1010010C9010010CB01001065
:10014000CD010010CD010010CD010010CD01001037
:10015000CD010010CD010010CD010010CD01001027
:10016000CD010010CD010010CD010010CD01001017
:10017000CD010010CD010010CD010010CD01001007
:10018000CD010010CD010010CD010010CD010010F7
:10019000CD010010CD010010CD010010CD010010E7
:1001A000CD010010CD010010CD010010CD010010D7
:1001B000CD010010CD010010CD010010CD010010C7
:1001C00000BE00BE00BE00BE00BE00BEEFF3058054
:1001D000103800BEF2EB887134B3001054B3001035
:1001E0003402001090A31AE700201F49086006C8D7
:1001F00081F3088810471D48006800282FD10DA4FE
:100200000ECC002902D000F012F8F9E71849194A7B
:10021000002000E001C19142FCD1174988471749ED
:1002200088471749884700BEFDE701C901C29A42C5
:10023000FBD3704754B30010C0000020F00B002027
:1002400084BE0010000004200000042084BE0010C2
:10025000001004200010042000000000704709482E
:1002600000F0B4FA0047000008ED00E0000000D004
:10027000F00B0020481D0220BD240010CD05001009
:100280007D2400105756000006005250ABB3605357
:100290007CA3001006005250861C03028CA30010A1
:1002A000060052505422A29D98A3001005005250FF
:1002B000DE65F46884BE0010F8B5C04606480749FC
:1002C000091A8B10C90FC91810B5491003D0044B77
:1002D000002B00D0984710BDF00B0020F00B002041
:1002E00000000000054B10B5002B03D00449054861
:1002F00000E000BFFFF7E2FF10BDC04600000000B5
:1003000008170020F891001010B504001F2100F01C
:1003100093FB00220021200000F0A6FB002120001A
:1003200000F0BCFB10BD0000D0231B061A69024977
:100330000A40DA61586170470018180070B5000370
:10034000214B1B685840E023DB0118401F4B18600D
:1003500007F096FFFA239B00C418002511E01C4B00
:1003600004221A60184B1B68DB05FBD5164B5B6833
:100370009BB2184A93420CD80135EDB2164B0022BD
:100380001A7007F07DFFA04218D2134B1B78002B88
:10039000E5D1114B1B78002BF3D10D4B04221A60D1
:1003A000094B1B68DB05FBD5074B5B689BB2094A11
:1003B0009342E6D9084B01221A70E2E7064B00226D
:1003C0001A70280070BDC04600C0044000D0044030
:1003D00000E00440AB0D00003E1D022010B50121DD
:1003E0000B4C2068494207F025FC0020FFF7A6FFD0
:1003F0000100084B180004F021F8206800230022B7
:10040000002107F0F5F90A2008F0B2F8E7E7C04646
:10041000FC120020F891001010B501210F4C20684B
:10042000494207F007FC0120FFF788FF0C4B1870CA
:1004300003F0BAFD0B4903F09CFD03F011FE02002E
:100440000B00094803F0FAFF206800230022002176
:1004500007F0CEF90A2008F08BF8DEE7FC12002046
:10046000411D02200000A0410892001010B5124B5F
:100470001C68124903F091FD03F0BEFD80B2A30099
:100480001B199B000E4A944663441A6842401204AA
:10049000120C802149010B431A600A4B1A68930021
:1004A0009B189B00634400041A685040000C000431
:1004B0001943086010BDC046F412002000409C455E
:1004C0000C000540F812002010B5012007F062FA78
:1004D000254B186008F0D4FD1B20FFF715FF1A20EC
:1004E000FFF712FF0B2000F0F1FA0C2000F0EEFAFB
:1004F000132000F0EBFA142000F0E8FAD0231B06DA
:10050000802212015A62802464015C6280221203FC
:100510005A62802252035A620421002000F08CFAB1
:100520000421012000F088FA104B00221A601049C3
:100530000A60104BFA2212015A605A600E4A1A6180
:100540001A611B680122100098430C4B186009685F
:100550008B005B189B0007498C46634419688A43EB
:100560001C43226010BDC046FC120020F412002083
:10057000F81200200000054087130000001005401D
:1005800070B584B000260396802464000B490C48A3
:1005900003AB0193012500950023220007F0F4FD31
:1005A00002960849084802AB0193009500232200F7
:1005B00007F0EAFD07F01AFE04B070BD20920010AB
:1005C000DD030010409200101904001010B504F073
:1005D000EFF8FFF779FFFA20C00001F000FB802060
:1005E0004001FFF7A1FEFE208005FFF73FFFFFF768
:1005F000C7FFFEE7034B1B6802201840431E9841CB
:10060000C0B2704700C0064010B5024800F032F892
:1006100010BDC046D419002010B5002901D0002318
:100620000AE0104B104A11481F3101F02BFF002245
:100630000DE03732C25401334A1E9A420ED90F2BB5
:100640000CD85A080A4CA45CDA07F0D404221441EE
:100650000F222240092AECDC3032EBE7C0180023DD
:10066000037010BD60920010AC92001068920010F0
:10067000D419002070B588B0040004AD002604969B
:100680000922002105A803F043FD0096092200215C
:1006900001A803F03DFD4B232B700D226946280075
:1006A00008F03AFD002304E05A1D69468A5CE254D2
:1006B0000133072BF8DD08B070BD0000EFF31080A8
:1006C00072B6034B1B68002BFBD0BFF35F8F7047E4
:1006D0002C0100D0BFF35F8F024B00221A6080F321
:1006E000108870472C0100D0F8B506000C001500EA
:1006F000FFF7E4FFE308F718F15C0722224001232B
:1007000093400B4205D1DBB20B433B70FFF7E2FF96
:10071000F8BD2100280001F04DFFF0B583B00600C0
:10072000019114001F00FFF7C9FF00E00134BC4233
:100730000CD8E308F518F35C0721214001228A4018
:100740001A42F3D1D2B21A432A7001E00124644262
:10075000FFF7C0FF002C02DB200003B0F0BD019BBF
:10076000002BF9D0089801F025FF0000002307E0D6
:10077000054A9A189200BFF35F8F00211160013380
:100780001F2BF5D97047C04640000034054A107849
:10079000431CDBB21370172B02D9130010221A70FE
:1007A0007047C046E80A002010B582B00100054C31
:1007B000054B00931F2318222000FFF7AEFF02B065
:1007C00010BDC046541200203494001010B5010032
:1007D00018231B8814221088984710BD10B50100FB
:1007E00018231B8816221088984710BDF0B5C646FE
:1007F00000B507000E0000250123984600E00135F2
:10080000B5420AD2AC003C192068FFF7DFFF206038
:100810000028F4D100239846F1E7404680BCB84652
:10082000F0BD0000F8B5DE4657464E464546E0B5F9
:1008300006000F0015000A9A934250D31A0E9246F2
:100840001B0298460A9A00234046514603F014F8CA
:1008500081467400A419A4002F4B9C46644463682D
:10086000834200D26060331FDBB29B46012B3CD930
:10087000C0239B012343802212011A60274BB20040
:10088000D158002907D0586902F0B8FF0130430061
:100890001B18033BFDD26D0123685D40E0222A4016
:1008A00080235B0123431A605A46012A28D98023FA
:1008B0009B012343802212011A604B4663604A4623
:1008C00000234046514602F0D7FF144BB600985122
:1008D0000120F0BCBB46B246A946A046F8BD104B6D
:1008E000104A1148332101F0CDFD012FC0D1C023A2
:1008F0009B01234303221A60A368DB07FCD5CAE7E8
:100900002168794003220A401A60A3680125BD408E
:100910001D42FAD0CBE7C0460080004058120020AC
:1009200050940010A49400106494001030B583B06B
:100930000C2001F0D5FCFFF75DFE00280DD0002350
:1009400004E02E4A99002E4888500133092BF8D92B
:100950002A4B2C4A5A6203B030BD2B4B00229A67B7
:1009600001F030FD294B01221A60274B5B6C012BF3
:10097000FBD1274B03221A60234B9B6B012BFBD12E
:10098000013300930433234A0121234801F018FC6A
:1009900005230093214A0121214801F011FC214B3C
:1009A0000093002202210420FFF73CFF1E4D00951A
:1009B0002B00002201210520FFF734FF104C00948A
:1009C0002300002200210720FFF72CFF00942300C2
:1009D000002200210820FFF725FF0A4B0093230087
:1009E000002200210920FFF71DFF00952B000022A7
:1009F00000210620FFF716FFADE7C0465812002081
:100A0000006CDC021BB70000008000403CB00040DE
:100A100030B00040002F685900800240008C8647AB
:100A200000C00240001BB70040597307014B800013
:100A3000C05870475812002010B58300084A9446E9
:100A400063441A684024624080341440802252017A
:100A500013431C60C000034B9C466044416010BDC2
:100A600004C001400040014080000B4B9C466044A4
:100A700000290DD00823002A0CD004221343026859
:100A800053400C221A4080235B0103431A607047D5
:100A90000023F0E70022F1E704C00140002909D05B
:100AA0008000094B9C46604480239B010343402205
:100AB0001A6070478000044B9C466044C0239B0131
:100AC000034340221A60F4E704C0014010B501233B
:100AD0008340D0221206936293610521FFF7ACFF99
:100AE00010BD0000074B9B68103080001950BFF309
:100AF0005F8FBFF35F8F044B0021196082F3108872
:100B00007047C04600ED00E0240100D010B5038816
:100B1000DA0A1C2A05D15B055B1502335B00C0189D
:100B200010BD034B034A0448B12101F0ABFCC046A1
:100B3000B49400102C970010CC94001010B5091A32
:100B40000B1F0A4A88180A4A904208D8C90706D4D7
:100B50005B105B055B0D0748184380B210BD064B68
:100B6000064A0748A32101F08DFCC046FC0700009F
:100B7000FE0F000000E0FFFF089500102097001016
:100B8000CC94001010B5091A04394A08090B08D191
:100B90004905490D064B0B430380064B1343438025
:100BA00010BD054B054A0648AB2101F06BFCC04661
:100BB00000F0FFFF00F8FFFF38950010F4960010DA
:100BC000CC94001001238340034A10681840431E50
:100BD0009841C0B27047C04600E100E0002904D04F
:100BE000034B1860034B18607047034B1860FBE71A
:100BF00080E200E000E100E080E100E010B50123C8
:100C000083401800FFF7EAFF10BD00000123834076
:100C1000014A13607047C04600E200E0024B9B6847
:100C200010308000C058704700ED00E010B5FFF7AD
:100C3000F5FF002805D0054BC01A2F2803D8012046
:100C400010BD0020FCE70020FAE7C046EC0A0020B7
:100C500070B504000D00EFF3108672B60C4B1B68E4
:100C6000002BFBD0BFF35F8F2000FFF7D7FF094BAE
:100C7000984201D0A84205D1320029002000FFF798
:100C800031FF70BD044B054A0548862101F0FAFB8F
:100C9000240100D0CD010010489500105497001099
:100CA000CC940010F0B5DE4657464E464546E0B5BA
:100CB00089B0814601911500EFF3108A72B66D4B31
:100CC0001B68002BFBD0BFF35F8F6B4B00269E573A
:100CD000002E41DB7400A419A400684824180622E1
:100CE000A256654B1A70664B9A684B4610339B00B0
:100CF000D35898461F00181A2F2839D9614B9845A8
:100D000030D105AF604B3B80604973009B4698191A
:100D100080005A4B984640440230FFF70FFF78801E
:100D20005B4BBB80FF23BB71FD71019B07933300BD
:100D30005B449B00434407CF07C301231C43A046E9
:100D4000524641464846FFF7CDFE09B0F0BCBB46CF
:100D5000B246A946A046F0BD4E4B4F4A4F48D72158
:100D600001F090FB4E4B4C4A4C48DE2101F08AFBCF
:100D700001380C2102F042FD002912D101239F43CA
:100D8000BB463B000027DA79AA4211D90621595601
:100D900000290CDB4A005218920038491F008B18BA
:100DA000F1E7404B3C4A3D48EA2101F06BFB1F0054
:100DB000002F2ED005AB3C4A1A80813A5A80062378
:100DC000FB560293002B17DA384805AB9B469880F8
:100DD000029A9A71DD71019A0792381D2100FFF77E
:100DE000ADFEB880BE71254B7200921992009B181F
:100DF0005A4613CA13C3A3E7381DFFF787FE010045
:100E00007000801980001D4BC0180430FFF796FE5B
:100E1000DBE705AF1C4B3B801C49730002939B1919
:100E20009B00164A90461A0042440392901CFFF71A
:100E300085FE7880039A101D5946FFF77FFEB88023
:100E40001B4B5A464146521A524153431B0DBB712C
:100E5000FD71019A0792029B9B199B00434407CFA7
:100E600007C3114B5A461380813B538001231C4317
:100E7000A04665E7240100D0421D0220EC0A0020B4
:100E800000ED00E0CD01001000A1FFFF1C0B0020D1
:100E900001BDFFFF809500103C970010CC9400101E
:100EA000A8950010D09500100148000001BD000079
:100EB000AAAA0000F0B5CE46474680B583B006002A
:100EC0000D00EFF3108872B64F4B1B68002BFBD060
:100ED000BFF35F8F4D4B9A6834001034A300D7588E
:100EE0004B4B9F4207D0AF4200D18BE00197494B5B
:100EF000FB1A2F2B09D9424639003000FFF7F2FDCB
:100F000003B0C0BCB946B046F0BD3000FFF75AFE92
:100F1000814600213000FFF771FEBFF35F8FEFF3D2
:100F20000581002901D08C4211D10123019C9C43F1
:100F30000020A368AB4212D00622A256002A0DDB85
:100F400053009B189B00334A2000D418F1E7324B22
:100F5000324A36213248FF3101F094FA2000AB4288
:100F600049D106256557002D2BDB2A4B6A00521903
:100F700092009B189A68A260DA79E2719B795BB261
:100F8000A371002B0FDA2748A080224B6A00521968
:100F900092009B18244A11789971157049463000C7
:100FA000FFF72CFEA7E7680040198000194BC01816
:100FB0000430FFF7ABFD0100231D1800FFF7BEFD55
:100FC000E2E7002912D100280ED0FF238371174BCE
:100FD000838015490B78A3710E4A154BA41A6441FE
:100FE00063431B0D0B70D9E7094FF2E71149201D30
:100FF000FFF7C8FDD2E7104B084A6A210848FF31C5
:1010000001F040FA024F76E7240100D000ED00E045
:10101000CD010010EC0A0020449600100C9700103F
:10102000CC94001001BD0000421D022001BDFFFF55
:10103000AAAA0000260B00207896001070B50122A5
:1010400002432E4BD31A2F2B28D8EFF30583002B06
:101050002BD0EFF3108C72B6294909680029FBD018
:10106000BFF35F8F254C274905002D1B6D41694358
:10107000090D4CB2244989689B00C95891421BD084
:101080000021032932D81D4B4A00521892009B18A8
:101090009B795BB2A3421FD00131F2E71B4B1C4A84
:1010A000C7211C48490001F0EDF91B4B184A922159
:1010B0001848FF3101F0E6F9134A92681749D150F8
:1010C000174B1A7882711C70BFF35F8F0C4B002294
:1010D0001A608CF3108870BD084B4A005518AD009B
:1010E0005D19FF26AE710F4AAA80E9E70E4B084A48
:1010F000D1210848490001F0C5F9C046EC0A00209A
:10110000240100D0AAAA000000ED00E080960010A3
:10111000D8960010CC940010A8960010CD010010B5
:10112000421D022001BDFFFFB49600100022044BB7
:1011300002E0044902C30132072AFAD97047C046C7
:1011400000E400E08080808010B582B00100074C90
:10115000074B0093052300222000FFF7DEFA00284A
:1011600001DB1F23181A02B010BDC046471D022024
:10117000BC960010024B9C46614489000160704798
:101180004000003410B5002B02DB0260436010BD4C
:10119000024B034A03483F2101F074F97097001095
:1011A000809800108C97001070B582B00600140073
:1011B0001D00FA22920000230698002102F0B6FEDC
:1011C00002000B0012196B41002B09DB6846FFF788
:1011D000D9FF009A019B32607360300002B070BD8D
:1011E00001225242004BF1E7FFFFFF7F10B582B0B2
:1011F000040000F073FD02000B006846FFF7C2FF19
:10120000009A019B22606360200002B010BD30B5DF
:1012100085B004000D0002A8FFF7E8FF029A039BC7
:1012200000952000FFF7C0FF200005B030BD10B5CD
:101230000400FFF7ABFA01002000FFF79BFF01233A
:101240005B426360BFF35F8F10BD10B50400FFF712
:101250009DFA01002000FFF78DFF01235B426360D0
:1012600000232372BFF35F8F10BD0000034B9C4629
:10127000614489000160BFF35F8F70474000003414
:1012800010B504000120FFF78FFA01002000FFF7DE
:10129000EDFF10BD084B5B6A994209D8064A926A75
:1012A000824207D2994201D0012002E0002000E0F2
:1012B000002070470120FCE70040054010B50029E0
:1012C0000AD003681B7B8B4206D38068054B9C4683
:1012D00061440901401810BD034B044A04483C21F5
:1012E00001F0D0F8FFFFFF0F98980010B49B00109A
:1012F000BC980010F8B504001700FFF7DFFF066880
:10130000456839002000FFF7D9FF026843680120D3
:10131000AB4201D802D00020C0B2F8BDB242FBD827
:10132000F9E7000010B5002B02DB0260436010BD3E
:10133000024B034A03483F2101F0A4F870970010C4
:10134000809B00108C97001010B582B004000498A8
:10135000059912184B41002B09DB6846FFF7E2FFA5
:10136000009A019B22606360200002B010BD012240
:101370005242014BF1E7C046FFFFFF7F10B5002945
:1013800008D0037B8B4205D300684B005B18033BFE
:10139000C01810BD024B034A0348682101F072F8DF
:1013A000F09800105C9B00100C99001010B5437B66
:1013B0008B4201D1012010BDFFF7E0FF8378002BA5
:1013C00001D10020F7E70120F5E770B50400857B27
:1013D000002D01D1280070BD2900FFF7CFFF437811
:1013E000A373002B00D1E373002383704370037059
:1013F000F0E70000F8B506000C001500FFF7BEFF8F
:101400000700002C0DD0002D11D0AC4215D02900C2
:101410003000FFF7B3FF84703B78002B13D13D7091
:10142000F8BD0A4B0A4A0B486F2101F02BF80A4B12
:10143000074A0848702101F025F8084B044A05487E
:10144000712101F01FF843703D70E9E754990010D5
:10145000389B00100C990010609900106C990010D6
:1014600070B506000D001400002914D0002A14D015
:10147000436880689847002806D022002900300081
:10148000FFF7B8FF280007E02A0021003000FFF72F
:10149000B1FF200000E0100070BD0800FCE7000074
:1014A00070B504000D1E0CD0FFF768FF0023837099
:1014B00043700370617B2A002000FFF7D1FF607347
:1014C00070BD034B034A0448A52100F0DBFFC04672
:1014D000849900104C9B00100C99001070B504000A
:1014E0000D1E0FD0FFF762FF00280BD1E17B002912
:1014F0000ED1A37B002B03D1E37B002B0DD1A57371
:10150000E57370BD084B094A0948F62100F0BAFF9F
:101510002000FFF733FF4570EBE7064B034A044812
:10152000FB2100F0AFFFC04688990010289B0010F7
:101530000C990010AC99001010B5002907D0036871
:101540001B7B8B4203D3C0680139401810BD034B8D
:10155000034A0448412100F095FFC04698980010C6
:10156000149B0010BC98001070B505000C0008001A
:1015700000F090FC0949200000F0D0FBFFF706F9CD
:10158000074B9C466044800068602C75D0231B0686
:101590001B786B75034BA400E55070BD85160010D9
:1015A000400000342817002010B582B0040000F07D
:1015B00095FB02000B006846FFF7B4FE009A019B02
:1015C00022606360200002B010BD70B584B00400DA
:1015D00016001D0002A8FFF7E7FF029A039B009682
:1015E00001952000FFF7B0FE200004B070BD0000A0
:1015F000F0B583B0070001921D000AAB1C780BAB5D
:101600001E78002C0BD000682100FFF7CFFE0028C9
:1016100009D0194B194A1A48672100F033FF0068B6
:10162000FFF7D3FE0400002C02D1200003B0F0BD70
:1016300021003800FFF742FE019B03604560089BD4
:101640008360099BC36038682100FFF729FFA0422F
:10165000EBD1387D019A2B0000F0A8FB051E01D0CC
:10166000002E04D00C9B002BDFD01D70DDE7386806
:10167000210000F055FDF5E7C0990010689B0010AF
:10168000BC980010F0B5DE4657464E464546E0B5DC
:101690008FB00B900021794B8200D458894683E0AB
:1016A00029002000FFF70AFE804602684368921B6B
:1016B000BB41002B09DD43461A685B680B9800F0BC
:1016C00075FB0023984600268AE0002B01D1002AF2
:1016D000F1D10021584600F019FD0700A84215D1AC
:1016E00043461A685B680892099343469E68DB6824
:1016F0009846002E10D029002000FFF71DFF037828
:1017000099461B021F432761002069E05C4B5D4A3C
:101710005D488E2100F0B6FE5C4B5A4A5A48922131
:1017200000F0B0FE2369002B00D177E0BB4219D155
:1017300006980799002342428B4100920193089A30
:10174000099B0CA8FFF700FE0C9A0D9B0021049149
:101750000131039102954146019100962000FFF767
:1017600047FF16E04A4B474A4748A12100F08AFE4E
:10177000069A079B002B01D1002A52D1206829002C
:10178000FFF7ACFE29002000FFF7D6FE03780133F7
:101790000370002323616268BFF35F8F13608AF3D5
:1017A00010880120002861D00CA8FFF7FDFE0C9ED8
:1017B0000D9F00220023089209936268EFF3108ABC
:1017C00072B61368002BFCD0BFF35F8F23689B4673
:1017D0005D7B002D00D063E70023984600260020A3
:1017E0006368BFF35F8F00221A608AF31088002EAF
:1017F000D8D04B461F022F4341463800B0470690D1
:1018000007916268EFF3108A72B61368002BFCD060
:10181000BFF35F8F079B002B00DA83E7079B002B4A
:10182000A6DD2369002BA9D0BB4219D10CA8FFF774
:10183000BBFE0C9A0D9B06980799009001910CA88D
:10184000FFF782FD0C9A0D9B002104910131039159
:1018500002954146019100962000FFF7C9FE98E7E6
:101860000B4B084A0848A42100F00CFE0FB0F0BC56
:10187000BB46B246A946A046F0BDC0462817002088
:10188000E8990010989B0010BC980010009A001076
:101890000C9A001010B5084B1A68EFF3108172B65D
:1018A0001368002BFCD0BFF35F8F034805F0B2FB39
:1018B0000020002110BDC046E01B002010B50C4BDD
:1018C0005B68002B04D00B480A21FFF753FC10BDC6
:1018D000074C094A20682300102100F082FB0320F6
:1018E00000F0F0F903212000FFF73EFEEBE7C046D1
:1018F000340B0020E01B0020F512001010B5064B41
:101900005B68002B01D0044810BD044B044A054815
:101910005E2100F0B7FDC046340B0020489A00104D
:10192000FC9A0010BC980010F0B5DE4657464E46B3
:101930004546E0B58DB0060090461F00169B9A46BE
:10194000179B994618AB1B780793272302AA944646
:10195000634400221A7021E001003000FFF7ECFD23
:1019600000783CE00698002B5CD0079B002B59D0F8
:101970004946D04704000D0003000B4359D000290D
:1019800040DB08A8FFF710FE089A099B0094019518
:1019900008A8FFF7D9FC089B9846099F7268EFF3E7
:1019A000108B72B6136859424B41D9B20691002B85
:1019B000F8D1BFF35F8F273302AA944663440493A0
:1019C0000023039302934B460193534600934246F0
:1019D0003B003000FFF70CFE0400051EBCD173680D
:1019E000BFF35F8F002119608BF31088002D17D093
:1019F000272302AA944663441B78002BB2D100022D
:101A00002043B0E700236242AB410092019342467B
:101A10003B0008A8FFF798FC089B9846099FBDE784
:101A2000012040420DB0F0BCBB46B246A946A046DC
:101A3000F0BD0698F6E7F0B5C64600B584B00500DF
:101A4000884616001F000AAB1C78FFF757FF029468
:101A5000019700962A004346FFF766FF04B080BC5A
:101A6000B846F0BDF0B5C64600B505000C1E42D024
:101A70004268EFF3108772B61368002BFCD0BFF3F7
:101A80005F8FE6B22B68984631001800FFF78EFC96
:101A900000282AD02B69A34213D0240AE4B23100D3
:101AA0002800FFF749FD0378A34211D000206B689E
:101AB000BFF35F8F00221A6087F3108880BCB8469E
:101AC000F0BD0E4B0E4A2C210E48FF3100F0DAFC1F
:101AD0003100404600F024FB0028E8D10A4B084AB8
:101AE00099210848490000F0CDFC2B69A342DED1C2
:101AF00000232B61DBE70020E0E7C0466C9A001072
:101B0000E49A0010BC980010909A001010B50400E0
:101B1000FFF7F4FE2100FFF7A5FF10BD407D7047E1
:101B200030B587B004000D00EFF30583002B20D102
:101B300096225242D31712196B418B4202D803D11D
:101B4000824201D90022002304A8FFF7EBFB02A880
:101B5000FFF72AFD02980399049A059B121A8B41FC
:101B6000002B0BDC08D02000290000F0C3F807B0E0
:101B700030BD114800F01EFD002AF4D00F4A049831
:101B8000059900230093FFF756FF00280DDAEAE7D6
:101B90000B4B1A68EFF3108172B61368002BFCD060
:101BA000BFF35F8F064805F0D3F904980599FFF756
:101BB00071FB0028ECD0D6E7949A0010951800101D
:101BC000E01B002000B583B002000B006846FFF761
:101BD000FCFC00980199FFF7A3FF03B000BD10B50E
:101BE000FA2292000023002102F0A0F9FFF7EAFF99
:101BF00010BD000030B583B005000C00EFF3058385
:101C0000002B0FD10B4A00230093FFF714FF00288D
:101C10000BDD20BFFFF77AFF28002100FFF73AFB1A
:101C200003B030BDFFF736FBFAE728002100FFF7CD
:101C300031FBF5E79518001070B5EFF3058010380B
:101C4000EFF3108C72B6194B1B68002BFBD0BFF35F
:101C50005F8F01221300834015494B6315490B60C8
:101C6000154909780C00C440224213D0104A546A26
:101C7000124A8500AA58944205D3114AAA580E4C1C
:101C80009943217007E00A4A031D9B009958995017
:101C9000002200E00022BFF35F8F044B0021196097
:101CA0008CF31088002A00D0904770BD280100D026
:101CB000004005403C700540461D0220EC1B002002
:101CC0003C11002010B50100024A034B1800FEF73A
:101CD0000BFD10BDC09B0010401D0220044B5B6A31
:101CE000034A906A1900536A9942F9D17047C04675
:101CF00000400540084B5B6A01E0074B5B6A8B4282
:101D0000FBD301E0044B5B6A8B4203D1024B9B6A1D
:101D10008342F7D37047C0460040054070B50400C9
:101D20000E00EFF3108572B61B4B1B68002BFBD027
:101D3000BFF35F8F002E1CD02000FEF76FFF174B04
:101D400083420BD019002000FEF782FF0121200002
:101D5000FEF754FF0123A340114A1360114BA40066
:101D6000E650BFF35F8F0C4B00221A6085F310889A
:101D700070BD0C4BA2000021D1500122A2400A49A3
:101D80000B7893430B7005492000FFF793F800216F
:101D90002000FEF733FFE4E7280100D0391C0010D3
:101DA000386005403C110020461D0220F0B5DE469B
:101DB00000B584B00400150001921E000293FFF7E5
:101DC0008DFF03958E4202D84ED185424CD9EFF358
:101DD000108B72B6274B1B68002BFBD0BFF35F8FB5
:101DE000254A17780125A540EBB23B431370234BDE
:101DF0005D63221D92000199D150214AA1000298F1
:101E000088501B6A2B4212D11C4B1B6C2B4208D0F2
:101E10000020BFF35F8F174B00221A608BF31088EE
:101E200023E0184B184A1948C52100F02BFBFFF797
:101E300055FF8E4214D802D1039B834210D80E4B1B
:101E40001B78BB420ED00D4B1D625D631F222240EA
:101E5000012393400E4A1360074B1F700120D8E7FF
:101E60000020D6E70120D4E7012004B080BCBB46A7
:101E7000F0BDC046280100D0461D022000400540AC
:101E8000EC1B0020E49B0010489C0010089C0010F4
:101E900080E200E0EFF3108C72B60B4B1B68002B56
:101EA000FBD0BFF35F8F01238340084A13620849C8
:101EB0000A789A430A70BFF35F8F034B00221A60BF
:101EC0008CF310887047C046280100D000400540C0
:101ED000461D022010B5002908D0037B8B4205D394
:101EE00000684B005B18033BC01810BD024B034A4F
:101EF0000348682100F0C6FAF0980010509D0010C9
:101F00000C990010F8B506000C001500FFF7E2FF71
:101F10000700002C0DD0002D11D0AC4215D02900A7
:101F20003000FFF7D7FF84703B78002B13D13D7052
:101F3000F8BD0A4B0A4A0B486F2100F0A3FA0A4B7E
:101F4000074A0848702100F09DFA084B044A0548EA
:101F5000712100F097FA43703D70E9E75499001041
:101F60003C9D00100C990010609900106C990010B5
:101F700070B506000D001400002914D0002A14D0FA
:101F8000436880689847002806D022002900300066
:101F9000FFF7B8FF280007E02A0021003000FFF714
:101FA000B1FF200000E0100070BD0800FCE770B534
:101FB00005000023437301338373037BC373012440
:101FC00006E021002800FFF785FF0134E4B24470E9
:101FD000297BA142F5D82800FFF77CFF002343703E
:101FE00070BD10B5017342608360FFF7E0FF10BD64
:101FF000F0B5C64600B505000C1E03D1200080BC1C
:10200000B846F0BDFFF766FF4678002EF6D03100E7
:102010002800FFF75FFF47780023984643702100B0
:102020002800FFF757FF4346437032002100280085
:10203000FFF79EFF040039002800FFF7D9FF0200D8
:1020400021002800FFF794FF0400D7E7F0B5C6464B
:1020500000B504000D001700002927D0FFF73AFF54
:102060004378002B28D18378002B2BD101782000D6
:10207000FFF7BEFF06008046002F0AD0E17B002953
:1020800026D1A37B002B03D1E37B002B25D1A573A5
:10209000E5734346002B26D129002000FFF71AFFE5
:1020A00000234370300080BCB846F0BD114B124A8B
:1020B0001248382100F0E6F9114B0F4A0F483A2137
:1020C00000F0E0F90F4B0C4A0C483B2100F0DAF924
:1020D0002000FFF7FFFE4570D3E70B4B064A074889
:1020E000422100F0CFF931002000FFF7F3FE00237A
:1020F0008370D1E7649C0010289D00106C9C001038
:10210000A49C0010CC9C0010AC99001070B5040089
:102110000A00457B2900FFF799FF6073280070BD16
:1021200070B506000C1E40D0437B8B4207D0FFF7F2
:10213000D1FE05008178002906D1002036E001217A
:10214000FFF7E4FF012031E03000FFF7C3FE017824
:10215000A1420DD03000FFF7BDFE4178A1420AD068
:102160000029F7D1124B134A13486B3100F08AF95A
:102170006B78037001E06B7843700023AB706B7079
:10218000012221003000FFF761FF0200717B8142D4
:1021900005D03000FFF7ECFE7073012006E0074B1E
:1021A000044A0548712100F06DF9002070BDC04659
:1021B000B4960010109D00106C9C0010F09C001054
:1021C000F0B5C64600B504000E0017001D003748E4
:1021D00001F014FB8046364BFA18364B9A4239D838
:1021E0000100380001F00AFB0200103A98235B005E
:1021F0009A4235D86B1E062B38D8069B013B062B1E
:1022000034D83F09474537D32D04069B1B031D4394
:102210002368002B36DB284B9C4244D080235B0193
:10222000264A1360264A1360264A92681900914391
:10223000FAD12660A060221DC0239B0113432122F6
:102240001A602268002AFCDAE56008221A6080BC65
:10225000B846F0BD1C4B1D4A1D48112100F012F973
:102260001C4B1A4A1A48192100F00CF91A4B174A4C
:1022700017481C2100F006F9184B144A1448232172
:1022800000F000F922683F231340B342C3D1A36892
:102290001B051B0D8342BED1E368EE22D202134020
:1022A000AB42B8D1D3E780239B01B9E7001BB7004D
:1022B00080E84BD380F8A93200C0024000E0004023
:1022C00000F0004000C000405C9D00107C9E0010AB
:1022D000BC9D0010F89D0010149E0010609E001020
:1022E00080239B000343014AD3627047008005406E
:1022F000024B1A68024B5A607047C0460017002014
:102300000080054010B5174B8022D2051A60164B8D
:10231000164A1A6000290AD0154BE022D2041A602E
:10232000002809D1124B802212061A6010BD0D4BF5
:10233000E022D2041A60F3E743011B1A9B0018182D
:1023400000010C4B186080235B04984202D3094BB8
:10235000094A1A60FFF7CCFF054B8022D2051A60AC
:10236000E4E7C04600B0054008200140FCFF010042
:1023700000A0054000170020FFFFFF0010B503007C
:1023800010000C4A8024E4051460002B0DD00122BB
:102390001343094A094CD461094C5C4014625162F0
:1023A00093620021FFF7AEFF10BD034B0022DA61FC
:1023B000F7E7C04600B0054000800540D3C007B035
:1023C0002D3FF84F064BAA2212011A602F22DA6025
:1023D000044B054A1A60024B5B68002BFBDA70471E
:1023E000004002400060024000B0FA00054B9842F5
:1023F00004D3054B984203D3002000E0002070472F
:102400000120FCE7C0010010CC010010044B9B68C8
:10241000103080001950BFF35F8F82F3108870472F
:1024200000ED00E0024B9B6810308000C058704700
:1024300000ED00E0F8B505000E00EFF3108772B66E
:10244000FFF7F0FF0400B04203D0FFF7CFFF0028F2
:1024500006D03A0031002800FFF7D8FF2000F8BD71
:10246000024B034A03482F2100F00CF8889E00100D
:10247000149F0010CC9E001000BEFDE710B5FFF7C2
:10248000FBFF000030B583B00D001900002A0BD00F
:10249000074B084C019200932B000200200001F032
:1024A000CDFF0120FFF7E8FF034B1A00F1E7C0461C
:1024B000349F0010449F0010409F001070B52B4BBC
:1024C0002B4A1A602B4B2C4A1A602C4B9A682A4BC9
:1024D0009343FAD12A4C01E008CC9847294B9C42FF
:1024E000FAD3FEF723FA234B274A1A60234B9B6843
:1024F000DB43DB01FAD1254B40229A675A671A6702
:10250000DA66234C09E0234B234A24488721FFF74E
:10251000B9FF2000FEF78BFE0834214B9C4209D204
:102520002368002BF5D0012BEDD12000FEF78DFEA6
:102530000C34F2E71B4DA9681B4CC022200001F0AF
:10254000EDFDAC60EFF30583002B00D000BEFEF77D
:102550000DF9FEF7EBFDFFF7B1F9144C01E008CCE3
:102560009847134B9C42FAD370BDC04600E0004030
:10257000BFCDFBFE00F00040FE7F3C0000C00040ED
:10258000D40B0020E40B0020FFFFFF0100F001400E
:10259000C40B0020749F0010F89F0010949F00103F
:1025A000D40B002000ED00E000000020E40B002030
:1025B000F00B00200FB400B583B0084801F00EFF07
:1025C000049B002B07D005A90191180001F016FF0C
:1025D000034801F003FF0120FFF74EFFD49F0010D6
:1025E000E49F001010B50148FFF7E4FFE89F0010DA
:1025F000704710B5002802D00B684968984710BD95
:102600000100002007E083001B185B00501C0860DD
:102610001078C01830380A681378303BDBB2092BC9
:10262000F1D97047F0B5DE4657464E464546E0B50F
:1026300083B093461F000C9B9A460D9C0E9B9946B7
:102640000F9B9B0703D0B8460F00060022E00192C3
:10265000A34688464E46B9460700B44207D2551CE9
:102660004B4641462020B84701342A00F5E73D009B
:102670004F465C46019B9B46B1464646B8463700EE
:102680002E0007E0013C551C5346185D43463900B7
:10269000B0472A00002CF5D135003E0047460F9B7D
:1026A0009B0707D4100003B0F0BCBB46B246A94656
:1026B000A046F0BDB0464E46B9462F005D46531BBE
:1026C000B342EFD2541C4B4641462020B84722006B
:1026D000F5E7F0B5CE46474680B585B094469846B6
:1026E0000C9D0D9C0EAB1B789946109A119B129E67
:1026F000B7071CD4002B0CD0F7070AD54F46002F84
:1027000002D10C37374204D0013B02E030272F556D
:102710000134944201D21F2CF8D9F70707D59C4207
:1027200005D21F2C03D830272F550134F5E7F706C3
:1027300012D5770505D4002C03D0944221D09C42B9
:102740001FD00F9A102A32D00F9A022A37D01F2C8E
:102750000AD830222A5501341F2C05D84A46002AAF
:1027600033D02D222A55013403960293019400950B
:1027700043466246FFF756FF05B0C0BCB946B046B7
:10278000F0BD621E012C10D00F9F102F0BD0140033
:102790000F9A102AD8D1B206D6D51F2CD4D85822D9
:1027A0002A550134D3E7023CCBE71400C9E7B2064F
:1027B000EED41F2CECD878222A550134C7E71F2C01
:1027C000D2D860322A550134C1E7720703D52B22D3
:1027D0002A550134C8E73207C6D520222A550134CC
:1027E000C2E7F0B5DE4657464E464546E0B593B0E3
:1027F00081468A46089209931CAB10CB1B789B46F6
:102800001E9D219B9846002C03D1102342469A43DB
:1028100090468023DB0046461E4042461A4212D0B4
:10282000002C22D000260EE03033D9B2771C0AAB40
:1028300099552900200000F0E1FFAC4216D31F2F6C
:1028400014D83E0004002900200000F0D7FFCBB2CE
:10285000092BE9D94246920605D54121C918C9B2CA
:102860000A39C9B2E2E76121F8E727004346069337
:10287000209B05931F9B049303955B46029301974E
:102880000AAB0093099B089A51464846FFF721FF7F
:1028900013B0F0BCBB46B246A946A046F0BDF0B5A9
:1028A000DE4657464E464546E0B597B00A900B9136
:1028B0000C929A46209B9946219F22AA13789B4608
:1028C000249B0993259C289B98464A463A4302D16B
:1028D0001032934398468022D20045461540434625
:1028E00013420AD04A463A4341D000252E005346AF
:1028F0000D934D46099B9A461BE02E0053460D93BF
:102900004D46099B9A4614E03033DAB2731C99465F
:102910000EAB9A55524623002800390000F0ACFF58
:10292000BC4226D819D04B461F2B1CD84E4605005A
:102930000F00524623002800390000F09DFFD3B25B
:10294000092BE1D94246920605D54122D218D2B2CE
:102950000A3AD2B2DAE76122F8E7AA45E3D94E464D
:102960000D9B9A4608E04E460D9B9A4604E00026D1
:1029700002E04E460D9B9A4643460693279B0593DD
:10298000269B0493099B03935B46029301960EAB2F
:10299000009353460C9A0B990A98FFF79AFE17B0CA
:1029A000F0BCBB46B246A946A046F0BDF0B5DE4637
:1029B00057464E464546E0B591B0804689460C9252
:1029C0009A461A9C1B9D22002B002000290001F032
:1029D000CEF9002800D0ECE001225242D44B200076
:1029E000290001F0BFF9002800D0E2E001225242A4
:1029F000D04B2000290001F09FF9002800D0D8E03A
:102A0000002200232000290001F096F9002800D0C0
:102A1000E4E0069407958023DB001E9A1A400D928D
:102A20001E9A1A4201D106231C93069807990200A8
:102A30000B000892099303000A00024300D1D9E079
:102A4000080D4005400DBC4EB44660440A03120B0D
:102A50001E00BA4B13431F0001F09CF9B84AB94B52
:102A600001F02BF9B84AB94B01F008F90890099127
:102A70000022B74B3000390001F0FBF8B54AB64BE5
:102A800001F01BF902000B000898099901F0F6F813
:102A900001F098F9834601F07DF906000F00AF4A76
:102AA000AF4B01F00AF90022AE4B01F0E7F801F05C
:102AB00089F90890AC4AAD4B3000390001F0FDF8BF
:102AC00006000F00089801F065F9A94AA94B01F02A
:102AD000F4F802000B003000390001F0CAF80600DB
:102AE0000F0002000B0001F0E8F80A900B91089B20
:102AF000A14A9446634400210022089109921B05D3
:102B000009930023089332003B003000390001F0A4
:102B1000B5F80E900F9132003B0000208021C905CE
:102B200001F0A7F806000F000022944B0A980B99B9
:102B300001F0A9F80022924B01F0A0F802000B006E
:102B40000A980B9901F09FF800228E4B01F096F83D
:102B500002000B000A980B9901F095F802000B0097
:102B60003000390001F08AF802000B000E980F992E
:102B700001F089F80022714B01F080F8089A099B56
:102B800001F09BF806000F0008960997069A079B2C
:102B900001F0E8F800282FD001235B429C46E34473
:102BA0000022774B3000390001F06DF80890099150
:102BB00022E01E9B04931D9B03931C9B0293009495
:102BC000019553460C9A4946404600F0FFF811B073
:102BD000F0BCBB46B246A946A046F0BD002100228B
:102BE00006910792069480231B069C46AC446346DC
:102BF000079310E700239B465B466333C62B20D820
:102C000004261E9B1B0528D5089A099B1900114311
:102C10000FD05D4A5D4B0698079901F09BF800289C
:102C20007AD000225A4B0698079901F085F80028BF
:102C300072D01C9B5B4506DD5A469B1A013B1C93D8
:102C400003E00526DDE700231C938023DB001E9AAA
:102C50001A431E92002600239B461D9B9E4265D26E
:102C60009F1B02231E9A1A400A921E9A134202D0F8
:102C7000002E00D000275B46002B07D0089A099B46
:102C80000698079900F0FFFF0690079100220023A5
:102C90002000290001F050F8002800D07CE03D4BD6
:102CA0001E9A1340049303971C9B0293069B079C58
:102CB0000093019453460C9A4946404600F086F82A
:102CC000002E00D183E71E9B9B0671D54525441C31
:102CD0005346020049462800C0475A46D317D21827
:102CE0005A4005230593013E0496002303930A33BB
:102CF00002935B46DB0F0193009253462200494644
:102D00004046FFF76EFD0A9B002B00D15FE70200F3
:102D100047460C9E1D9D53E01C9B002B9DD00D9B98
:102D2000002B9AD01C9B013B1C9396E7002798E749
:102D3000FFFFEF7FFFFFEFFF01FCFFFF0000F03F11
:102D4000FB799F501344D33FB3C8608B288AC63F9A
:102D50000000F83F61436F63A787D23F71A37909F1
:102D60004F930A400000E03F1655B5BBB16B0240DF
:102D7000EF39FAFE422EE63FFF03000000002C4030
:102D800000002440000018402D431CEBE2361A3F9F
:102D900080842E41FFF7FFFF069C079D220029003B
:102DA00080200006844661440B000692079376E774
:102DB00065258CE7541C534649462020B84722001D
:102DC000931BAB42F6D3100001E7C046F0B5DE46D8
:102DD00057464E464546E0B595B006900791934656
:102DE0009946209F1E9A1F9B1000190000F0BFFFFC
:102DF000002831D101225242BF4B1E981F9900F08A
:102E00009BFF002837D101225242BC4B1E981F99CC
:102E100000F0A8FF00283DD10022B94B1E981F9951
:102E200000F0A0FF002850D10022B64B1E981F9939
:102E300000F082FF002848D1002200231E981F992D
:102E400000F07AFF002850D100239846229B5B05B2
:102E500000D4B6E0002458E0229B0393219B029308
:102E600003230193A84B00934B465A4607990698B3
:102E7000FFF7D8FB0EE1229B0393219B02930423CF
:102E80000193A24B00934B465A4607990698FFF7C9
:102E9000C9FBFFE00423229A1A4022990B4210D06A
:102EA0009B4B002A0FD00422229903912199029171
:102EB000019200934B465A4607990698FFF7B2FBDA
:102EC000E8E0944BEDE70322EEE7229B0493219B7D
:102ED000039302971E9B1F9C009301944B465A46F6
:102EE00007990698FFF762FDD4E01E9A1F9B002009
:102EF000002100F0BEFE1E901F9101239846A5E719
:102F00000CAB30221A55013F01341F2C01D8092F78
:102F1000F6D81E981F9900F055FF050000F03AFF03
:102F200002000B001E981F9900F0A3FE7A4BFA00D6
:102F30009B181A685B680A920B9300F0BEFE08901B
:102F4000099100F063FF060000F020FF02000B0073
:102F50000898099900F08DFE0890099100226F4BA6
:102F600000F000FF00282ED00136300000F00EFFE8
:102F700002000B000A980B9900F0E4FE002801D033
:102F800001350026002F2CD1280000F003FF02009D
:102F90000B001E981F9900F06CFE06000F00002227
:102FA0005E4B00F0C9FE002846D100225B4B30008A
:102FB000390000F0D7FE00283ED1EB073CD50135A3
:102FC0003AE0062746E70022544B0898099900F09A
:102FD000B3FE0028D6D1002E01D0F307D2D501369A
:102FE000D0E7AA461F2C11D8013F0A21300000F07B
:102FF00005FC651C30310CAB19550A21300000F07E
:10300000FDFB092E0ED906002C00EBE755461F2CC0
:103010000CD87B1E002F09D00CAA302111551F009F
:103020000134F4E72B0055461C00F0E71F2C03D8B1
:103030000CAB2E221A5501341F2C10D80A2128005F
:1030400000F0B4FB661C30310CAB19550A21280086
:1030500000F0ACFB051E01D03400EDE73400032383
:10306000229A1340012B1CD01F2C06D84346002B5C
:1030700032D00CAB2D221A550134229B0393219B95
:10308000029301940CAB00934B465A46079906985D
:10309000FFF7C8FA15B0F0BCBB46B246A946A04639
:1030A000F0BD219B002B13D04346002B02D10C33E3
:1030B00013420FD0219B013B2193190003E00CAB7D
:1030C00030221A5501348C42CED21F2CF7D9CBE7CF
:1030D0002199F8E72199F6E7229B5B0704D50CAB11
:1030E0002B221A550134C8E7229B1B07C5D50CAB10
:1030F00020221A550134C0E7FFFFEFFFFFFFEF7FEB
:1031000065CDCD4165CDCDC114A0001018A0001033
:1031100008A0001010A00010C0A100100000E03FA7
:10312000F0B5DE4657464E464546E0B593B082467A
:10313000884693461193002900D106E300255646A0
:10314000119B1878002800D102E3252809D06C1CB7
:103150005B462A004146B047119B0133119325007D
:10316000EEE701331193002720E001231F430132D2
:103170001192012418E002231F430132119201240D
:1031800012E004231F430132119201240CE00823B2
:103190001F4301321192012406E010231F43013224
:1031A0001192012400E00024002C09D0119A137818
:1031B000203BD9B21029F6D88B00C449CB589F4682
:1031C000119B1A781300303BDBB2092B10D92A2A45
:1031D00013D00B94119B1A782E2A1ED0119A1378B3
:1031E000683BD9B2122959D88B00B949CB589F46B0
:1031F00011A8FFF705FA0B90ECE71C9B1A1D1C9217
:103200001B68002B04DB0B93119B01331193E1E747
:10321000022217435B420B93F6E78022D20017434A
:103220005A1C11925A781300303BDBB2092B0BD990
:103230002A2AD3D11C9B1A1D1C921C68002C08DB67
:10324000119B01331193C9E711A8FFF7D9F90400C5
:10325000C4E70024F4E780235B003B43511C119139
:1032600051786C2901D01F0018E0C0239B001F4338
:103270000232119212E080233B43511C119151788C
:10328000682901D01F0009E0C0231F4302321192B8
:1032900004E080235B001F4301321192119B1878D8
:1032A000672816D8252826D30300253BDAB2422A00
:1032B00021D89300874AD3589F4680239B001F4301
:1032C00001321192EAE780235B001F430132119221
:1032D000E4E778280FD869280DD30200693AD2B202
:1032E000012393407C4A13420FD11A0600D507E20E
:1032F0005B0500D594E16C1C5B462A004146B04753
:10330000119B0133119325001AE778280AD062280F
:103310003AD06F283BD058283CD010239F43063B1F
:103320009C4601E010239C46582836D0692803D0DB
:10333000642801D00C2297437A0501D501229743D6
:1033400069282DD064282BD0BA0500D5A2E0FA0553
:1033500000D5C3E07A0600D4D5E01C9A111D1C915B
:103360001168FF220A4005970B9B04930394634660
:1033700002930023019300925B462A0041463000ED
:10338000FFF72FFA05002AE002239C46CCE708232A
:103390009C46C9E710239C46C6E720221743C5E791
:1033A000BA0520D4FA0550D47A0666D51C9A111DA8
:1033B0001C911168FF220A40D0171118414005974F
:1033C0000B9B0493039463460293D20F01920091E6
:1033D0005B462A0041463000FFF703FA0500119BC7
:1033E00001331193ACE61C9A073207218A4311007E
:1033F00008311C91116853689946DB170C930D93A3
:103400000C9A0D9B100048400E904A4653400F9373
:103410000E980F990C9A0D9B801A99410E900F915E
:1034200008970B9B07930694634604930023059328
:103430004B46DA0F0292009001915B462A0041460A
:103440003000FFF72CFA0500C9E71C9A111D1C91EA
:103450001268D0171118414005970B9B04930394F1
:1034600063460293D20F019200915B462A004146C7
:103470003000FFF7B6F90500B1E73A0605D51C9A0A
:10348000111D1C910023D25E96E71C9A111D1C9100
:10349000126891E71C9A073207218A43110008310C
:1034A0001C9108970B9B0793069463460493002393
:1034B0000593029353681268009201935B462A00B9
:1034C00041463000FFF7EBF9050088E720A0001027
:1034D00064A00010B0A00010419000001C9A111DC3
:1034E0001C9105970B9B049303946346029300235E
:1034F0000193136800935B462A0041463000FFF7B2
:1035000070F905006BE73A0606D51C9A111D1C914F
:1035100012681204120C26E71C9A111D1C911268E5
:1035200021E7462819D01C9B0733072293431A0032
:1035300008321C9204970B9A039202941A685B68F3
:10354000009201935B462A0041463000FFF73EFCA3
:103550000500119B01331193F2E520231F43E2E79D
:10356000672801D0472802D180231B011F4345282B
:1035700001D0472801D120231F431C9B073307227A
:1035800093431A0008321C9204970B9A03920294F8
:103590001A685B68009201935B462A00414630003E
:1035A000FFF704FA0500119B01331193C8E50223CC
:1035B0001A003A4091463B421DD001241C9B1A1D23
:1035C0001C926F1C18785B462A004146B0474B4658
:1035D000002B14D1119B013311933D00B0E5571C12
:1035E0005B4641462020B04723003A005C1C9D42C8
:1035F000F5D81500E2E701232A000B9DF6E73A0013
:10360000B1460B9E06E0571C5B4641462020C8474A
:103610002C003A00651CA642F5D817004E46D9E7A3
:103620001C9B1A1D1C921B689A46002C25D1012256
:103630005242534601E001330A001978002902D0B2
:10364000511E002AF7D152469B1A8022D20039001F
:1036500011408946174202D0A34200D9230002221A
:103660001100394010913A4209D02A0025005746EE
:103670009A4633004E46994621E02200D9E72A00B7
:103680004546A04606E0541C5B4629002020B04772
:103690003B0022005F1C0B999942F4D84446A8468F
:1036A0003B00250057469A4633004E46994606E0B1
:1036B0001D000137541C5B464146C847220038783C
:1036C000002804D0002EF4D06B1E002DF0D1150080
:1036D00053464E46109A002A03D1119B0133119391
:1036E0002EE50B9F2A0006E0551C5B464146202034
:1036F000B04723002A005C1C9F42F5D81500ECE778
:1037000021233B431C9A111D1C9112680593082329
:1037100004930394083302930023019300925B46C1
:103720002A0041463000FFF75CF80500119B013389
:10373000119305E56C1C5B462A0041462520B047E5
:10374000119B013311932500FAE40B4B9A46F5E4E3
:10375000B2465D450DD35B465A1E5B46414600208E
:10376000D047280013B0F0BCBB46B246A946A046DD
:10377000F0BD2A00F1E7C046F125001000B585B084
:103780000290039101210448009313004A4202A9C8
:10379000FFF7C6FC05B000BDF32500100148042169
:1037A000014B1847600B0020ED070010124A936F81
:1037B0009B0815D29066D166002905D0FFE7FFE788
:1037C000FFE7516F106F704704B580210906C217DB
:1037D0005140002800D0C84305F0C6FC002104BDBC
:1037E000F0B5146E556E576F166FFFF7E3FF146652
:1037F000556657671667F0BD000000D0114A936FF9
:103800009B0813D210665166002905D0FFE7FFE739
:10381000FFE7516F106F704704B5002801D00020FA
:10382000C04305F0A1FC002104BDC046F0B5146EF4
:10383000556E576F166FFFF7E5FF146655665767AD
:103840001667F0BD000000D094464A4A926F920875
:10385000624601D228E0C046F0B5464E346E756E21
:10386000776F366F00F020F89446424A146655662A
:10387000576716676246F0BD94463E4A926F9208BB
:10388000624601D254E0C046F0B53A4E346E756ED1
:10389000776F366F00F04CF89446364A14665566DA
:1038A000576716676246F0BD002B24DB11D0002954
:1038B0003EDA00B5C943404200D1013100F038F88A
:1038C000C943404200D10131DB43524200D10133B0
:1038D00000BD002AEBD1002801D1002905D000202D
:1038E000C90FC90701D1C043410800B505F024FC48
:1038F0000022002300BD00B500290ADBDB43524251
:1039000000D1013300F014F8C943404200D1013125
:1039100000BDC943404200D10131DB43524200D1D6
:10392000013300F005F8DB43524200D1013300BD02
:10393000002923D1002B18D1002A0CD0BC460D4FF2
:1039400038667A6600210023FFE7FFE7FFE77A6F1A
:10395000386F67467047002801D00748010000B55E
:1039600005F0EAFB0022002300BD02000B0000204E
:1039700000217047000000D0FFFFFFFF002B00D0A8
:10398000BFE0130C28D1002AE7D080B4114F39666C
:103990007A66FFE7FFE730B4040C7B6F396F1B04D6
:1039A00023433B667A66FFE7FFE7FFE7C04684B242
:1039B0007B6F3D6F1B0423433B667A66FFE7FFE79F
:1039C000C04600232C042D0C7A6F386F0019694112
:1039D000B0BC7047000000D0F0B594460025140E2E
:1039E00001D112020835140F01D112010435940FD0
:1039F00001D192000235D40F01D152000135D40B10
:103A00000134254F7C66254C3C660E0C93B2FFE7D3
:103A1000FFE7FFE73C6F6643360C7703BE46734310
:103A2000DF0B5B04C01AB941130C7343DB18C91ACE
:103A3000CE086643360CB64493B273431F0F1B0186
:103A4000C01AB941130C73431F0B1B05C01AB941AF
:103A5000860D8F023E436643360C092D24DB520A45
:103A60007243801A7703460A6643360C16235B1BA3
:103A7000DE40DF40BF1964466643821B7046043552
:103A800006330100D940A840C01900D30131A24239
:103A900006D20023F0BD0000000000D0FFFFFFFFB2
:103AA000121B0130F3D3F1E709277F1BFE40644668
:103AB000A2B27243801A00D20139220C7243130C55
:103AC0001204821A99410B00704604351337010025
:103AD000F940A840801900D30131002B02D1A24245
:103AE0000AD2F0BD013000D30131121BFAD2013BE2
:103AF000F8D1A24200D2F0BD013000D30131121B37
:103B0000F7E7F0B51C0C00D080E00CB400251C0ACF
:103B100004D11B02160E3343120208351C0B04D1CC
:103B20001B01160F3343120104359C0B04D19B007B
:103B3000960F334392000235DC0B02D192185B41A1
:103B400001351C00971864410134464F7C66464C91
:103B50003C660E0CFFE7FFE7FFE7C0463C6F66439D
:103B6000360C7703BE4697B27743C01B00D20139AB
:103B7000C01B00D201399FB27743C91BC91B170C68
:103B800077437E04FF0B801BB941CE086643360C99
:103B90000C2D33DBB644120B1F053A431B0B97B2B7
:103BA0007743C01B00D201399FB27743C91B170C62
:103BB00077433E043F0C801BB941860D8F023E4384
:103BC000664329277F1BFE400C3D7746AF40BF1957
:103BD00030BCA2B2ABB272437343801A9941220C3B
:103BE0007243130C1204801A994102000B00013732
:103BF000001BA941F9D2781E0021F0BD0C277F1BC4
:103C0000FE4077467F0BAF40FF19E0E700245D1CC4
:103C100007D0144F7D663966FFE7FFE7FFE7FFE750
:103C20003C6F95B29EB265436643401BB141150C93
:103C30001E0C6543664336042F0C3E432D04401B87
:103C4000B141994204D202000B0020000021F0BDD6
:103C500001D19042F7D3801A994101349942F2D3AD
:103C6000F6E70000000000D0FFFFFFFF48404140A2
:103C7000484018B4134B5B68019308BD18B4114B4E
:103C80001B68019308BD94460F4A926F920805D2B3
:103C9000624618B40B4BDB68019308BD0A4AF0B5C5
:103CA000146E556E576F166F6246FFF7F2FF064AA5
:103CB0001466556657671667F0BD18B4014B9B68CC
:103CC000019308BDDC190020000000D0FFB5504072
:103CD0004240504059404B40594000E0FFB5154F1D
:103CE0004C00640D03D0BC4204D10C0314D8002056
:103CF000090D09055C00640D03D0BC4204D11C030E
:103D00000AD800221B0D1B0501264B4009D44B404D
:103D100003D58B4200D18242FFBD9942FCD1904233
:103D2000FFBD0B43DB1803431343F5D0C9434918C8
:103D3000FFBD0000FF07000000B5FFF7CFFF804187
:103D400000BDC04600B5FFF7C9FF01D9002000BD86
:103D5000012000BD00B5FFF7B9FF01D9002000BD6B
:103D6000012000BD00B5FFF7B1FF804100BD01207B
:103D700040054A00121804D85A00121801D8002031
:103D80007047012070470020704700000021002884
:103D900005D17047C1174840401AFAD0C90713B57A
:103DA000064B1B6898470CBC441CA2401005120B24
:103DB0000349091B09051943114310BDDC1A0020F2
:103DC0001F04000010B54C00620D8023D218DB00E8
:103DD000D21A5B057E2A10DD9E3A13DACC1709034E
:103DE000490819435242D140640001341532202A57
:103DF00005DAD0400843604310BD002010BD0846DE
:103E0000604310BDC80FC018013810BD18B4024B74
:103E10005B6A019308BD0000DC19002010B5014861
:103E2000FEF7C8FB10A2001070B513231C78012CFC
:103E300012D0012C12DC214B214A93642148FCF75B
:103E4000C5FC214B186070BD20491D4A9800815067
:103E500001331F2BF8D9ECE70023FAE71C48FCF7E5
:103E6000BDFC05001B48FCF7B9FC023803789B0039
:103E70007F2B09DD12488022290000F04FF9022C27
:103E800008D0022CDADCD6E7134B144A144832214E
:103E9000FEF7F8FA134B1A88B5231B029A4209D190
:103EA000114B1A88114B9A4204D1114B1A88114BAD
:103EB0009A42E6D00020FEF77DFBC046F93E001096
:103EC000DC1900204C330000DC1A00201D3E0010DD
:103ED000534400005346000028A20010C4A2001062
:103EE0007CA2001054380000D83800004946000079
:103EF0009C3800005946000007B56046002800D1F4
:103F000000BE01880A0A0230DF2AFAD1C9B282084B
:103F100004D3028840880004104300E00068024A8D
:103F20005050039007BD0000DC190020514343436B
:103F3000C9188C46110C83B24B4310B4040C614376
:103F400092B280B2504362431C041B0C001910BC97
:103F500059411304120CC0185141614470470000CC
:103F60004840414048400E4B5B6818470C4B1B686B
:103F700018470C4A936F9B0802D2094BDB6818471D
:103F8000F0B5146E556E576F166FFFF7F6FF054AC2
:103F90001466556657671667F0BD014B9B68184756
:103FA000E01A0020000000D0491A002808D1084675
:103FB00070470000C10FC90700D54042002817D044
:103FC000F44603B40B4B1B68984706BC81409E38EF
:103FD0004042803107D20B0607D04900490AC0058C
:103FE0001043084360470130F8E7490A8902F5E7C2
:103FF00070470000DC1A002041000A0E80231B06D7
:104000007E2A0BDD9E3A0BDAC117400240081843A6
:104010005242D04049000131484370470020704768
:10402000C00FC01801387047C0420DD300B5400022
:104030004008002100F00EF8002801D4404200BDE5
:104040008020000600BD0000014BDB69184700001E
:10405000E01A0020014B5B6A18470000E01A0020BC
:10406000014BDB6F18470000E01A002010B5014833
:10407000FEF7A0FA409F001070B513231E78184871
:10408000FCF7ACFB0500012E11D0012E09DDAB1EA3
:104090001B789B007F2B1DDD12488022290000F039
:1040A0003DF81148FCF792FB104B186070BD0D48AD
:1040B0005422290000F032F8002300E001331F2BC6
:1040C000E3D8084A9C00A258002AF7D10849054ABB
:1040D000A150F3E7074B084A08484221FEF7D2F9FE
:1040E00053460000E01A00204C330000DC1A002088
:1040F0006D400010D8A2001050A300100CA30010B7
:1041000001480421014B1847700B0020ED070010F7
:10411000014B1B6818470000700B0020014B5B68C7
:1041200018470000700B002010B5030008001100B4
:104130001B68984710BD0000F8B507000D00160079
:10414000437D002B02D0002400200CE00368110006
:10415000280098472DE03B7D10E03B681548022180
:104160009847601C0134B44214DA002CF3DD2B199B
:10417000013B1B780D3B5A425341DBB22A5D0A2AB0
:10418000F0D1002BEED1A042E7DA3B68211A2818C3
:104190009847E2E7B04203DA3B68311A281898479B
:1041A000002E06DDAD19013D2B780D3B5A425341DF
:1041B0003B75F8BDC8A3001070B505000368002B5F
:1041C00016D00C4B1C6805E0290004C92000FFF73D
:1041D000B3FF2469002C09D02368002BF9D0064BCB
:1041E0001B68002BF0D0A342F3D1EDE700232B6036
:1041F00070BDC046E8120020F012002070B5050026
:104200000C000B68802B05D023685A1C2260E41830
:10421000257170BD0800FFF7CFFFF5E710B5002B43
:1042200002DB0260436010BD024B034A03483F219A
:10423000FEF728F970970010CCA300108C9700109F
:1042400010B582B00400FDF749FD02000B0068467E
:10425000FFF7E4FF009A019B22606360200002B038
:1042600010BD000070B582B0060014001D00FA22D7
:104270009200002306980021FFF758FE02000B0071
:1042800012196B41002B09DB6846FFF7C7FF009A44
:10429000019B32607360300002B070BD0122524257
:1042A000004BF1E7FFFFFF7F30B585B004000D0044
:1042B00002A8FFF7C5FF029A039B00952000FFF7B5
:1042C000D1FF200005B030BD00B583B0FA218900D0
:1042D0006846FFF7E9FF009A019B024804F06CFF73
:1042E00003B000BDCC0B002010B5024804F01CFF49
:1042F00010BDC046CC0B0020F0B5CE46474680B579
:1043000083B006000D0090461C00FFF7DDFF8146DC
:104310006B1C05D0002C08D0194F1A4B1C6807E005
:10432000300004F0C7FE0500F4E7174FF5E72469F5
:10433000002C17D02368002BF9D0144B1B68002BDE
:1043400001D0A342F3D12A0031002000B8474346F0
:10435000002BECD06B46D91D0A230B7001222000E4
:10436000B847E4E74B46002B07D16B1E9D41E8B2EE
:1043700003B0C0BCB946B046F0BDFFF7B5FFF4E7E7
:1043800029410010E812002039410010F0120020ED
:10439000094A01E010331A001368002B08D0834249
:1043A000F8D1002907D1036913600023036102E0FB
:1043B000002900D010607047E812002010B5064BAD
:1043C0001C6801E098472469002C03D06368002B27
:1043D000F8D1F8E710BDC046E812002070B505001E
:1043E00004F068FE04000023012201002800FFF70A
:1043F00083FFFFF7E3FF200070BD000070B5A2B09F
:1044000004000E00FFF760FF0500002301930A4837
:104410003300220001A9FFF7B1F9040001A8FFF75A
:10442000CBFEFFF7CBFF002D02D1200022B070BDE4
:10443000FFF75AFFF9E7C046FD4100100FB400B581
:1044400083B004A901C90191FFF7D8FF03B008BCEC
:1044500004B0184770470000014B00221A707047E3
:10446000431D02204B79FF2B0CD18B79002B0BD1F4
:10447000CB79012B0AD1082A0AD98A78054B1A7000
:10448000092000E0002070470020FCE70020FAE748
:104490000020F8E7431D02200120704770B504009A
:1044A0000D000348FCF792F903002900200098470B
:1044B0005542000010B5012926D1117953791B020C
:1044C0000B43124909788B4201D000201DE053783C
:1044D000012B03D0022B10D0002016E09178D37866
:1044E0001B021943DB0506D54B0A012098407F23A8
:1044F0001940FFF7D3FF0020F9E7642200210020D4
:10450000FDF73CFF012000E0012010BD431D02200B
:104510000123037000487047E4A3001010B50A7827
:104520004B781B0213438A7812041A43CB781B067C
:1045300013439622D200934200D010BD0021080000
:10454000FFF7ACFF024B1860024B19607047C04682
:104550004C1200205012002010B5002B02DB02602C
:10456000436010BD024B034A03483F21FDF78AFF19
:104570007097001070A400108C97001010B582B0D6
:104580000400FDF7ABFB02000B006846FFF7E4FFF9
:10459000009A019B22606360200002B010BD000001
:1045A00070B582B0060014001D00FA2292000023AC
:1045B00006980021FFF7BAFC02000B0012196B41AC
:1045C000002B09DB6846FFF7C7FF009A019B3260AA
:1045D0007360300002B070BD01225242004BF1E71F
:1045E000FFFFFF7F30B585B004000D0002A8FFF784
:1045F000C5FF029A039B00952000FFF7D1FF200022
:1046000005B030BD10B582B00400049805991218A9
:104610004B41002B09DB6846FFF79EFF009A019B88
:1046200022606360200002B010BD01225242014BA3
:10463000F1E7C046FFFFFF7F10B5024B1878FCF78B
:10464000E5FA10BD441D02200268EFF3108172B636
:104650001368002BFCD0BFF35F8F416070470000F0
:1046600070B50F4B1B68002B16D00D4C2000FFF7C8
:10467000EBFF0C4B00221A7021686368BFF35F8F59
:104680000A6083F3108800240025074B1878FCF794
:10469000BDFA2000290070BDFA24A4000025F4E72B
:1046A00020170020451D0220441D0220F0B587B0D0
:1046B000040016001D000EAB1F7804A8FFF75EFF74
:1046C000049A059B0096019504A8FFF79BFF049AA6
:1046D000059B02970D9901910C9900912000FDF71F
:1046E00023F907B0F0BDF0B5C64600B584B00500AB
:1046F000884616001F000AAB1C78FDF7FFF80294ED
:10470000019700962A004346FFF7D0FF04B080BC13
:10471000B846F0BD10B582B01948002104F02CFD58
:10472000002822D1174B1B68002B26D0154C2000E7
:10473000FFF78AFF144A137801214B40DBB20121B5
:10474000117021686268BFF35F8F0020086082F3F8
:104750001088002B11D00D4A012300930023FA206A
:1047600080000021FFF7BFFF07E001200021404249
:1047700001F036F8024804F0D7FC02B010BDC04684
:10478000E41B002020170020451D02206146001078
:1047900010B5054B1868002804D0044B1968002296
:1047A00000F048FD10BDC0464C1200205012002001
:1047B00010B582B0D0231B061C68FDF79FF8FDF7EB
:1047C000ADF9A0422CD1234B1B7801F0D7FC224835
:1047D000FCF72DFD0120FCF7B7FC204C2070204990
:1047E000FF231840FCF734FA20780121FCF706FA81
:1047F0000520FCF71BFA041E18D01A4900220520D8
:10480000FCF750FAFBF7C2FF0100174B1800FCF74A
:104810002DFD16480121FFF7BBFD200002B010BDA1
:10482000134B144A1448B221FDF72CFE134A0123FE
:1048300000930023FA2080000021FFF754FFC443B7
:10484000E40F094808220021FFF762FC002CE4D0A5
:10485000DFE7C04650B30010E41B0020441D0220D7
:10486000154700103946001020170020800B00204B
:104870007896001060A40010FCA3001061460010A0
:1048800010B5002001F0A4F910BD000030B583B0D0
:1048900004000D00FFF7F4FF002830D0002001F0E5
:1048A000B3F900282ED0FA2189006846FFF79AFE56
:1048B000009A019B164804F07FFC002825D0FFF7E2
:1048C000DFFF002804D0002001F09EF900280CD161
:1048D00001200021404200F083FF032464420C4881
:1048E00004F022FC200003B030BD2A00210000208B
:1048F00001F096F9041EF2D103246442EFE7032489
:104900006442EFE703246442ECE703246442E9E7EE
:10491000E41B0020F0B5C64600B582B080460D000D
:10492000FA2189006846FFF75DFE009A019B2C483A
:1049300004F042FC002803D102B080BCB846F0BDB0
:10494000FFF79EFF002849D1264B00200021186068
:104950005960234804F0E8FBEEE7012000214042C3
:1049600000F03EFF002001F06FF9FFF789FF0028FB
:10497000EFD0002001F0E0F9002820D0AC42E8DAC6
:104980002E1B002001F0D8F90200864200DC320024
:10499000002AE2D043461919002001F0B1F90600BF
:1049A00001200021404200F01BFF002001F04CF9E3
:1049B000A419FDF793F90B4B18605960DEE7FDF77A
:1049C0008DF9084B1E685F68074A002392197B41E6
:1049D0009942BED8D2D19042D0D9BAE70024CDE7CF
:1049E000E41B0020F00C002020A1070000487047C5
:1049F00020A5001000487047CCA4001010B504009A
:104A0000154B1B78002B0ED0002C11D1134B144AE0
:104A10005A80012301335B009BB21048C0229200F0
:104A20001343038010BD0C481121FBF7F5FDEBE7A4
:104A3000052C0ED80B4BA400E4580023122BE9D808
:104A4000E15C0029E6D00133044A58008152DBB210
:104A5000F4E70020E6E7C046001C0220C012002058
:104A600009040000B4A4001002007F201040D20905
:104A7000400080184001014BC0187047001300200F
:104A800010B5038B3F333F229343022915D0124CBC
:104A90002268C260D31823609C0610D10F4C62407C
:104AA000634080246401A3420FD889061143802308
:104AB0001B060B434268136010BD5B00E7E7084B21
:104AC000084A09485421FDF7DDFC084B054A064811
:104AD0005621FDF7D7FCC0460417002000001050F7
:104AE00034A500104CA6001064A50010B8A5001055
:104AF000F8B505000E001400FFF7B6FF7F232B402A
:104B0000EF0985707A427A4142700022C2700683B2
:104B1000C476012F0DD0DA0012498C4662448260BF
:104B2000826800211160002B09D143600E4BC360E5
:104B3000F8BDDA000D498C4662448260F0E7012F2F
:104B400009D0013BDB000A4A9446634443602100DC
:104B5000FFF796FFECE7013BDB00064A944663440F
:104B60004360F4E7840010500001105080001050A2
:104B70000C0010500800105070B584B006000D00F5
:104B800014000C22002101A8FFF7C2FA6B461E7127
:104B900003236A4653710295210001A804F0FCFA30
:104BA00004B070BD70B50C001500FFF75DFF2A0062
:104BB000210000F00DF970BD10B5002804D10121CD
:104BC0000520FCF71BF810BD034B044AD52104480F
:104BD0004900FDF757FCC04600A600103CA6001097
:104BE00064A5001010B5002805D100220021802006
:104BF000FFF7D8FF10BD034B034ADB2103484900F0
:104C0000FDF740FC00A600102CA6001064A50010C3
:104C1000024B80225202DA647047C04600201150D5
:104C200070B5041E26D100F0ADF8164D0C23AB670D
:104C30001549FF220520FCF735F8144840220021D1
:104C4000FFF766FA002240210020FFF751FF002203
:104C500040218020FFF74CFF04F076FA01232B64FB
:104C600080239B05EB649023094AEA502000FFF75C
:104C7000CFFF70BD074B084A86210848FF31FDF77A
:104C800001FCC04600001150210400200013002048
:104C900010D0010000A6001060A6001064A500104E
:104CA0000B785B0602D14B78052B00D070478A78D1
:104CB000014B1A60FAE7C0460000115010B50A0017
:104CC00000280DD18878097953791B020B435B05C5
:104CD000590DD2789207920FFFF70AFF012010BDFD
:104CE000034B044AFC210448FF31FDF7CBFBC046CF
:104CF00000A600101CA6001064A5001010B504F05A
:104D000023FA10BD10B50400080011001A00002C91
:104D100003D1FFF747FF012010BD034B034A0448AE
:104D20000449FDF7AFFBC04600A600100CA600101A
:104D300064A500100A02000010B508004B0605D15A
:104D4000CB09012B0AD00222054B9A66FFF78CFE95
:104D500080221201002104F047FA10BD0122F3E77E
:104D60000020115010B508004B0600D110BDFFF710
:104D70007BFE0023C3700022014904F035FAF5E7F9
:104D8000FFF7FFFF10B580235B040C4A13600C4A49
:104D900013600C4B9A6880235B049343F9D10A4C4F
:104DA0009C2200212000FFF7B3F98022520100214C
:104DB0000648FFF7ADF90923636710BD00E0004026
:104DC00000F0004000C000400000115000001050F2
:104DD00070B504000D001600837E002B17D1A6824B
:104DE0000023E3820133A3762561200004F0DCF97F
:104DF000002804D0094A902380218902D150200044
:104E000004F0AAF9002805D00123237770BD04F02F
:104E1000E3F9E4E7200004F0D7F9F7E700201150A8
:104E200070B5050000240CE062001219D200184B86
:104E30001B689B18002B2AD05B6828009847013418
:104E4000E4B2144B1B78A34210D3134A002A0BD0B0
:104E5000A342E9D8E31ADBB2002B18D15A00D318C9
:104E6000DB000E4A9B18E7E72300F5E70C4C5322C2
:104E700000212000FFF74CF9E01C1022FF21FFF772
:104E800047F9200013302022FF21FFF741F970BDC0
:104E9000F80C00203C1D022011450010F0A7001066
:104EA000201000200268EFF3108172B61368002B07
:104EB000FCD0BFF35F8F4160704710B5FFF7B0FFC4
:104EC00000F0E4FD10BD70B505000C001600C868C8
:104ED00000F0E6FDE368320001212800984770BD2C
:104EE000F0B5DE4657464E46C0B582B00090013957
:104EF000C8B2FFF77FFD002800D18EE043789A46C4
:104F0000022B00D08BE0C5796C1101224A4B144072
:104F1000240119781026B14321431970AD112A409C
:104F20005201C9B22024A1430A431A70070009376D
:104F30008278C3781B021343C418A74266D27B78D9
:104F40000B2B09D001239B467B78042B6ED1E31BEE
:104F50009BB29946002538E0FB789B463B78FF18CA
:104F6000F2E76B005B19DB00344A1668F618002E76
:104F70003DD1002054E02B0032E0B268304B9A4221
:104F800042D1D34640E02C49CB18DD700132D2B279
:104F9000934509D9BB789B18DBB22749C918C97852
:104FA000FF29F0D000203BE026482B00019E320074
:104FB000390001F06FF9B4466744234B1B78AB42CC
:104FC000BBD200202CE00135EDB21F4B1B78AB4269
:104FD000F3D31E4A002ACED0AB42C2D8EB1ADBB2C2
:104FE000002B25D15E00F618F600194BF618B368B1
:104FF0004A4639000098984701900828E3D981452E
:10500000E1D35B46012BB8D00022C1E7114B002B46
:1050100010D000E000BF012002E0002000E00020EE
:1050200002B0E0BCBB46B246A946F0BD0020F7E79F
:105030000020F5E70120F3E720100020F80C002005
:10504000555E0010331000203C1D02201145001059
:10505000F0A700100000000070B505000C00CB7830
:1050600088780F2B50D89A002E498A589746FFF718
:10507000BDFC020012232100280000F0D3FC44E014
:10508000294B002B42D000E000BF021E40D08178A7
:10509000C3781B020B432100280000F0C3FC34E05E
:1050A000022B09D0214B002B34D000E000BF0200BE
:1050B000002A05D1002028E0FFF79CFC0200F7E75A
:1050C0009178D3781B020B432100280000F0AAFC42
:1050D0001BE02379617909021943FFF78FFC021E57
:1050E0001AD003782100280000F09CFC0DE0104B42
:1050F000002B13D000E000BF021E11D00378210066
:10510000280000F08FFC00E0002070BD0020FCE7CC
:105110000020FAE70020F8E70020F6E70020F4E797
:105120000020F2E764A7001000000000000000006B
:1051300000000000024B5878431E9841C0B27047EF
:1051400020100020024B18784007C00F7047C0465F
:1051500020100020034B1878FF38431E9841C0B23E
:105160007047C046BC0B002070B50400FFF7F2FF8B
:10517000061E01D0300070BD244853220021FEF7E6
:10518000C7FF234D2800FCF752F8224B1D60224D2B
:105190002800FCF775F8143D280001F0CFFB1F4BE9
:1051A0001D601F4B002B04D01E48FFF7B1F91E4BAA
:1051B000186000250BE06A005219D2001A4B1B68D8
:1051C0009B18002BD6D01B6898470135EDB2154BC4
:1051D0001B78AB4210D3124A002A0BD0AB42EAD85C
:1051E000EB1ADBB2002BC5D15A00D318DB000F4AF3
:1051F0009B18E8E72B00F5E70D4B1C702000FFF72C
:105200000FFD2000FFF7D8FC0126B3E72010002097
:10521000D80F002074100020B40B0020781000205C
:10522000114500103C1D0220F80C0020F0A70010D2
:10523000BC0B0020F0B585B007000E00150001ACD6
:105240000C2200212000FEF763FF08236370029701
:1052500003962900200003F09FFF05B0F0BD000079
:1052600070B50C00094B1D788B7870221A4201D062
:10527000002070BD064B9978200000F0CFFF002879
:10528000F7D021002800FFF719FDF2E7BC0B002042
:1052900020100020F8B5CE46474680B581460C0068
:1052A00017001E00089B9846002504E0099A137019
:1052B0002378E4180135AF4214DD6378052B16D14D
:1052C000E1788907890FB14213D121004846FFF7E1
:1052D000C7FF002807D0A378DA09012AE6D04246A2
:1052E0001370E5E70120C0BCB946B046F8BD002008
:1052F000F9E70020F7E7000010B57F200840C90952
:10530000400040183030044BC0180330034B19687C
:1053100000F040FF10BDC046201000207410002097
:1053200010B57F200840C909400040183030044BB8
:10533000C0180330034B196800F054FF10BDC0467D
:105340002010002074100020F8B5CE46474680B5E6
:10535000194800787F250D40CE09184C6F00E419DC
:10536000A4193034E478E40704D50020C0BCB94661
:10537000B046F8BD114CE419A4193027B946A14430
:105380004C46E4780127BC4667463C4327004C4620
:10539000E770FFF7B7FC0028E8D1084B6D005B19F8
:1053A0009B193033DA7801218A43DA70DA780331D5
:1053B0008A43DA70DAE7C046BC0B002020100020D8
:1053C00070B50F4B18787F240C40CD090D4B62004F
:1053D0009B185B193033DB789B0700D570BDFFF756
:1053E000ABFC084B64001B195B193033DA780221DF
:1053F0000A43DA70DA7801210A43DA70EEE7C04630
:10540000BC0B00202010002070B50F4B18787F24B3
:105410000C40CD090D4B62009B185B193033DB78D3
:105420009B0700D470BDFFF79DFC084B64001B195F
:105430005B193033DA7802218A43DA70DA7801397D
:105440008A43DA70EEE7C046BC0B00202010002033
:105450007F220A40C909044B52009B185B18303365
:10546000D8788007C00F704720100020F0B5C646DE
:1054700000B582B005000C00002000F011FB22787E
:1054800060231340602B00D185E1402B0FD02278A0
:10549000D206D20E012A00D1C9E0022A00D10FE1C2
:1054A000002A11D0002002B080BCB846F0BDC54B28
:1054B000002B00D171E1180000F0F2FA2200012166
:1054C000280000E000BFEEE7202B0AD0002B00D020
:1054D00069E16378092B00D967E19B00BA4AD35888
:1054E0009F4623790F2B00D959E1B84AD318DB78AE
:1054F000B74A002A05D0B74A127893420ED39B1AB6
:10550000DBB2002B00D04CE15900C918C900B24BE6
:10551000C91822002800FFF7D6FCC4E75A00D318A8
:10552000DB00AE4A1168C9180029F2D10020BAE7A1
:10553000200000F0BBFAA1782800FFF753FBA34A34
:10554000137802210B4313700120ACE79F4B5B786B
:105550006A460632137001232100280000F062FA27
:105560000120A0E7A678994B5B78DBB2B34205D067
:10557000964B5B78002B09D1002E13D1934B5E70B4
:105580002100280000F03AFA01208CE72800FFF7FC
:10559000B5FB8E4FBB7898462800FFF741FC434689
:1055A000BB70E9E731002800FFF79AFC0028E5D13D
:1055B00079E721002800FFF74FFD74E7A278E37830
:1055C0001B021343012B01D000206CE77F4A1378A4
:1055D00008210B4313702100280000F00FFA01206E
:1055E00061E7A278E3781B021343012B01D000206E
:1055F00059E7764A137808218B431370210028005D
:1056000000F0FCF901204EE7704B1A78510992081E
:1056100001230B4002210A4013436A4606321380DD
:1056200002232100280000F0FDF901203BE7237947
:105630000F2B00D9BBE0654AD318DB78644A002AF7
:1056400005D0644A1278934225D39B1ADBB2002B13
:1056500000D0AEE05900C918C9005F4BC91822003C
:105660002800FFF730FC002800D01CE723786022D8
:105670001A4200D017E763780A3B012B00D912E7E2
:1056800000F00EFA63780A2B0FD02100280000F0FA
:10569000B5F9012007E75A00D318DB004F4A11681B
:1056A000C9180029DBD10020FDE66B469A1D0023B6
:1056B000137001332100280000F0B4F90120F2E654
:1056C00021797F200840CE0970220A4273D13F4AD7
:1056D000400012189219D27C3D48002805D03D4860
:1056E0000078824212D3121AD2B2002A15D1560083
:1056F000B618F600384AB618002B10D0002E5CD031
:10570000220031002800FFF7DEFBCCE650008218B3
:10571000D20032480668B618EEE70026ECE7637858
:10572000012B12D0032B10D0002B01D00020BAE6A1
:105730002800FFF78DFE6B469A1D10800223210082
:10574000280000F06FF90120ADE6A078E27812029F
:10575000024304D1012B1AD02800FFF731FE002E9E
:105760002DD0220031002800FFF7ADFB002000F013
:1057700097F9164B34229B5CDB07D80F002B00D027
:1057800091E62100280000F039F901208BE628007D
:10579000FFF73AFEE3E7002085E6002083E60020DD
:1057A00081E600207FE600207DE600207BE60020E9
:1057B00079E6002077E6002075E6002073E60120F8
:1057C00071E6C04600000000A4A7001020100020D1
:1057D000114500103C1D0220F0A70010F80C00201D
:1057E00030B585B000F0CFFC002808D105B030BD41
:1057F00001AC2078FFF761FB2279594B9A70594B25
:105800001C6820001430FFF74DFB01A9200001F0B7
:1058100038F86269A369BFF35F8F0021116083F3D9
:1058200010880028E2D001AB5B78082BE7D89B00FA
:105830004D4AD3589F4601AB1878FFF73EFB4B4BC0
:10584000002BDCD000E000BFD9E7454B1A780124DB
:1058500001210A431A703322995CA1439954995C3F
:105860000420814399540132995CA1439954995C75
:105870008143995401AB187802A9FFF7F7FD00287E
:10588000BDD101AC20780021FFF756FA20788021A5
:10589000FFF752FAB3E701AB19797F220A40CC092E
:1058A0002F4B50001B181B193033D8780125A84303
:1058B000D870D8780335A843D870002A1CD0284B5C
:1058C00052009B181B19DB7C294A002A05D0294A63
:1058D0001278934217D39B1ADBB2002B00D085E7D6
:1058E0005A00D318DB00244A9B181C6901A842798E
:1058F000039B0078A04782E701A84279039B0078C8
:1059000000F0E2F87BE75A00D218D2001B4B1B686C
:105910009B18002BE9D169E7114B1B78DB0700D4FA
:105920006DE7174B002B00D169E70D4B1878000786
:10593000C00F00E000BF62E7094B1B78DB0700D413
:105940005DE7104B002B00D159E700E000BF56E7A0
:10595000029B002B00D152E7039898474FE7C046BF
:105960002010002078100020CCA7001000000000BC
:10597000114500103C1D0220F0A70010F80C00207B
:10598000000000000000000010B50023CB56002BE3
:1059900005DB802100230022FFF7D6FC10BD00218B
:1059A000F8E70000F8B50500124B9F89DE89B91BA6
:1059B00089B20B1C402900D940239CB20D4B1B78A7
:1059C0005BB2002B08DB0021B74211D00A4A23004A
:1059D0002800FFF7B9FCF8BDB74201D18021F3E7F9
:1059E000044B996804482200FEF798FB8021EBE7FE
:1059F0000022ECE7C40F0020E00F002070B5060085
:105A00000D00074C08222000FEF788FB0023A3604E
:105A1000E381A38129003000FFF7B6FF70BDC046C7
:105A2000C40F0020F0B5C64600B580460C00160035
:105A30001D00154B08221F001800FEF76FFBBE600B
:105A40000023FB81A379E179090219430B1CA942C8
:105A500000D92B1C99B20C4A9381A279E3791B02DD
:105A6000134309D0002901D0002E0AD04046FFF789
:105A700099FF80BCB846F0BD21004046FFF784FF87
:105A8000F7E70020F5E7C046C40F002010B5034833
:105A900014220021FEF73CFB10BDC046C40F0020BD
:105AA000014B18617047C046C40F002010B50100BB
:105AB000044C08222000FEF731FB0023A360E381A1
:105AC000A38110BDC40F002070B505001C00C909DA
:105AD000294B1B78DB098B4211D0002C47D1274B77
:105AE000002B02D02449FFF7DBF8234B1B69002B66
:105AF00003D0214A032128009847012070BD1E4B86
:105B00001B785BB2002B07DB1B4B9868002830D05A
:105B10001B492200FEF702FB174AD389A1B25B188A
:105B20009BB2D381916809199160D288934201D0C8
:105B30003F2C18D8104B1B69002B05D00E4A0221B0
:105B400028009847002804D00B492800FFF71CFFC5
:105B5000D4E700212800FFF7EFF880212800FFF7A5
:105B6000EBF80120CAE72800FFF71CFFC6E700207A
:105B7000C4E70020C2E7C046C40F0020A14C0010BB
:105B8000E00F002070B5040005001035280000F07B
:105B900062FE3F2801D8002070BDE1780020FFF7A9
:105BA000ABFB0028F8D0280000F055FE3F2808D9AC
:105BB00092239B00E218E17840230020FFF7C4FB0A
:105BC000EAE7E1780020FFF7ABFB0020E4E7000004
:105BD00010B50400FFF7AEFA002801D1002010BD77
:105BE000FFF7B0FA002809D1064BB22292006243B7
:105BF0009B181B79DB0703D50130F0E70020EEE7A7
:105C00000020ECE7FC0C002010B5B2239B004343BE
:105C100010330248181800F0EEFD10BDFC0C0020F7
:105C200070B5B2239B005843064BC51892B2103092
:105C3000C01800F047FE04002800FFF7A3FF200073
:105C400070BDC046FC0C002070B50500FFF772FA6D
:105C5000002804D10023002B09D1002070BDFFF7DC
:105C600071FA002801D10123F5E70023F3E7B224FC
:105C7000A4006C432034214BE4180434200000F0CD
:105C8000BAFD002801D10020E8E71C4BB2229200A7
:105C90006A439B1899780020FFF72EFB002801D15A
:105CA0000020DBE7B226B6006E43A2239B009C4691
:105CB0006644124BF61840223100200000F002FE2C
:105CC000041E0ED00D4BB22292006A439B189978A5
:105CD000030032000020FFF737FB00280CD0200023
:105CE000BCE7064BB22292006A439B1899780020C9
:105CF000FFF716FB0020B1E70020AFE7FC0C002007
:105D000070B50500B224A40044432034094BE418C4
:105D1000043492B2200000F00CFE0600200000F0D7
:105D20006AFD3F2801D8300070BD2800FFF78CFFC6
:105D3000F9E7C046FC0C002010B5B2239B00584385
:105D40002030034BC018043000F085FD10BDC04664
:105D5000FC0C0020F0B5CE46474680B583B02A48FB
:105D6000B22292000021FEF7D3F90027002F04D0C1
:105D700003B0C0BCB946B046F0BD234EB224A40067
:105D80007C433519FF236B71002398461F4AEA8034
:105D900001222A81AB72EB7208232B732100383168
:105DA0008919F83399462000103080194346009332
:105DB00001334A4600F0E1FC21003931FF318919F5
:105DC0002000203080190430012300934A4600F05F
:105DD000D4FC8E239B00E3189946B1444846FBF758
:105DE00026FA4346EB614B462B6290239B009C4670
:105DF0006444A4192000FBF71AFA2C6343466B6332
:105E00000137FFB2B2E7C046FC0C002000C2FFFF22
:105E100070B50025002D00D070BDB224A4006C43E5
:105E20000B4EA01905220021FEF772F92000103058
:105E3000801900F083FD2034A4190434200000F000
:105E40007DFD0121200000F098FD0135EDB2E1E774
:105E5000FC0C0020F0B583B004004B79022B4ED12E
:105E60008B79022B4FD10023002B01D0002547E076
:105E70002848B225AD005D4340198078002802D043
:105E80000133DBB2F0E7234BEE188B7833700F78D9
:105E9000CF19092503E03B785D19ADB2FF187B7877
:105EA000242B01D19542F6D9052B09D07B78042B00
:105EB00002D17B790A2B10D03000FFF763FE1FE080
:105EC00039002000FFF7CCF900281ED0BB78737092
:105ED0003B785D19ADB2FF18E8E739784D19ADB2DE
:105EE0007918B31C0193F31C0093022302222000B3
:105EF000FFF7D0F900280AD00E35ADB2DCE7002557
:105F0000280003B0F0BD0025FAE70025F8E70025DA
:105F1000F6E7C046FC0C0020F8B5140012786023A8
:105F20001340202B00D07FE0444A0025002D00D0F4
:105F30007CE01678277963791B023B439E4206D0AA
:105F40000135EDB2B2239B009C466244EEE76378D4
:105F5000222B31D009D8202B11D0212B03D101299C
:105F600023D0012061E000205FE0232B05D101292F
:105F700049D003294CD0012057E0002055E00129E9
:105F800003D0032908D001204FE006320723210067
:105F9000FFF748FD012048E0294B002B48D0911D18
:105FA0002800FEF7BBFA01203FE00632072321005C
:105FB000FFF738FD012038E0012903D0032906D07E
:105FC000012032E02100FFF719FD01202DE0A1782A
:105FD000E3781B020B430120190001400E005C080E
:105FE000044013714B425941C9B22432100000F0F1
:105FF000C4FC144B002B1DD022003100280000E00F
:1060000000BF012011E02100FFF7F8FC01200CE0A7
:106010000D4B002B10D0A378E1780902194328001A
:1060200000E000BF012000E00020F8BD0020FCE7F8
:106030000120FAE70120F8E70120F6E7FC0C002038
:106040001D4500100000000000000000F0B5D6461D
:1060500000B582B001900F0000930024002C0ED0F8
:10606000002C00D07CE0EB78BB4216D0AB78BB4272
:106070004DD00124200002B080BCBA46F0BDB2254C
:10608000AD006543394BED18EB78BB42E8D0AB78F7
:10609000BB42E5D00134E4B2E0E710239A46AA44BB
:1060A00092239B00E9186B461A88504600F041FC89
:1060B0002F4B002B1BD06B79FF2B18D0002600E054
:1060C0000136009B9E4212D26A79AB199221890057
:1060D0008C4663441B789A42F2D1504600F0A0FBF4
:1060E0000028EDD16979200000E000BFE8E7214BEE
:1060F000002B04D0504600F093FB002803D028006A
:10610000FFF740FDB2E72000FEF742FBF7E71A4B2E
:10611000002B02D0200000E000BF2000FFF794FD1C
:10612000002801D00124A5E72800243000F063FBFB
:10613000002817D1009B002B16D09E0601D0012409
:1061400098E7A9780198FFF7D7F8041E01D1012438
:1061500090E7A978002300220198FFF7F5F889E776
:10616000002487E7012485E7012483E7FC0C002055
:1061700000000000914700100000000010B5002052
:10618000FEF7F2FF10BD10B5FEF7E4FF002800D0C7
:10619000012010BD70B504000D000378DB07D80F97
:1061A000002B1DD123785B07DE0F002B19DB0121AB
:1061B0004942280002F0E8FF2378DB07DA0F002BC2
:1061C00007D123785B0709D4237804221343237073
:1061D0000126280002F0A8FF300002E01600F8E7D0
:1061E000002070BD70B506000C000121494220005E
:1061F00002F0CAFF33785B07DD0F002B04DB2000C1
:1062000002F092FF280070BD3378DB0704D43378A6
:10621000042293433370F2E70025F0E702794379D3
:106220001B0213435B055B0DC2789207920F022A93
:106230000FD0032A19D0012A01D00020704702296B
:1062400004D0134A9A421AD30120F7E78022D200E1
:10625000F8E7022903D0402B15D80120EEE7802271
:10626000920093420DD10120E8E7022904D0402298
:106270009A420AD30120E1E78022D200F8E7002009
:10628000DCE70020DAE70020D8E70020D6E7C046A8
:10629000FF03000030B58A1801E00C78091991421B
:1062A0000AD24C78052CF8D18D787A342C406400D1
:1062B0000419ED096355F0E730BD03008A1890B268
:1062C000814202D85A00904203DB5B009BB2C01AA5
:1062D00080B2704770B505000800AC889A420BD3B5
:1062E000D11A89B200291ED08C4210D2944209D80A
:1062F000121B93B26B810AE0D11A89B26600891928
:1063000089B2EFE7A21893B2F4E71B1B9BB29C4241
:10631000FBD92968EA885204520C5343C918FDF787
:10632000FDFE012070BD0020FCE770B582B00500C5
:10633000160093080CE00A784B781B0213438C7804
:1063400024041C43CB781B0623432B600431030039
:10635000581E80B2002BEED1033332001A401E4289
:1063600001D102B070BD0023019301A8FDF7D6FE54
:10637000019B2B60F5E7F0B5DE4657464E46454695
:10638000E0B583B005008A460CA909788488E01A34
:1063900080B21C1B1419A4B2EF887F047E0C070086
:1063A0007743BFB27443A4B2A3462C68A04673439C
:1063B0009844002908D001291AD003B0F0BCBB468C
:1063C000B246A946A046F0BD904205D3724341466D
:1063D0005046FDF7A3FEF0E73A0041465046FDF770
:1063E0009DFE2968380050445A46FDF797FEE4E7C1
:1063F000904206D3724392B241465046FFF795FF52
:10640000DBE703233A009A43914641465046FFF7A3
:106410008CFF42464A440323380018401F4230D0C4
:1064200004231B1A9BB2191C5B4500D95946CFB2F5
:10643000FF230B405946CC1AA3B29B46002301937D
:1064400001AB04E010781870013308000132411EDE
:10645000C9B20028F6D1296804E008781870013321
:10646000170001317A1ED2B2002FF6D1019B52469D
:1064700013605B46002BA0D05A465046FFF755FFED
:106480009BE72968F5E7F0B5C64600B582B01E0067
:1064900008AB1B8809AC277884889E420FD3F51A75
:1064A000ADB2002D1FD0AC4205D2B44210D8331B80
:1064B0009BB24381250095420FD315000DE0F51ADC
:1064C000ADB2A8466500AC4645466544ADB2E8E7C6
:1064D000A619B3B2EDE71B1B9BB29C42FBD90097F8
:1064E0002A00FFF748FF280002B080BCB846F0BD84
:1064F000F0B583B004000D0016001F0000690028ED
:1065000003D00121494202F03FFE23899BB26289F8
:1065100001970092320029002000FFF7B4FF050028
:10652000618989B2A0882A00FFF7C7FE60812069CF
:10653000002801D002F0F8FD280003B0F0BD70B5CE
:1065400082B01600950809E00B6803701D0A4570BB
:106550001D0C85701B0EC370043025006C1EA4B288
:10656000002DF1D1032332001A401E4201D102B0A6
:1065700070BD0B68019301A9FDF7D0FDF7E7F0B5F9
:10658000DE4657464E464546E0B583B005008A468E
:106590000CA90878AC88E11A89B21C1B1419A4B2A2
:1065A000EF887F047E0C0F007743BFB27443A4B220
:1065B000A3462C68A04673439844002808D00128BD
:1065C0001AD003B0F0BCBB46B246A946A046F0BD07
:1065D000914205D3724351464046FDF79FFDF0E7D7
:1065E0003A0051464046FDF799FD2868390051446C
:1065F0005A46FDF793FDE4E7914206D3724392B207
:1066000051464046FFF79BFFDBE703233A009A43DE
:10661000914651464046FFF792FF42464A440323C3
:10662000380018401F422ED004231B1A9BB2191C9D
:106630005B4500D95946CFB2FF230B405946CC1ACF
:10664000A3B29B4653461B68019301AB04E0187844
:106650001070013308000132411EC9B20028F6D182
:10666000286804E0197801700133170001307A1EA0
:10667000D2B2002FF6D15B46002BA2D05A4651462B
:10668000FFF75DFF9DE72868F5E7F0B585B00600E8
:106690000391151E029300D16DE0C068002803D05D
:1066A0000121494202F070FD3489A4B2718989B296
:1066B000F379DB091AD1B3888C420FD3611A89B2FE
:1066C0008B4211D95B1A9BB22F1C9D4200D91F1C13
:1066D000BFB2002F47D0B288230035E0611A89B2DB
:1066E0005A00891889B2EBE70023EDE7B788AF427B
:1066F0000ED8029B002B21D1ED1BF3885B045B0CB1
:106700006B43039A94469C44634603930C00E0E772
:106710008C420DD3631A9BB25B197A0093420FDB54
:106720007A1B92B23800FFF7C8FD04002F00D0E7B3
:10673000631A9BB27A009B189BB2EDE70C00C8E786
:106740002F00C6E79B1A9BB29A42FBD9029A00928D
:106750003A0003993000FFF712FFB0883A00210099
:10676000FFF7ABFD3081F068002801D002F0DCFCBF
:10677000380005B0F0BD1700FAE7F0B583B00400AB
:10678000019116001D0008AB1F7880231B029A425E
:106790002DD8C068002803D00121494202F0F4FC42
:1067A0002069002803D00121494202F0EDFC019B41
:1067B0002360A6806D046B0CE588ED0BED031D4393
:1067C000E580FB01E2797F2717401F43E771002333
:1067D00063812381E068002801D002F0A5FC2069D4
:1067E000002806D002F0A0FC012003B0F0BD00207C
:1067F000FBE70120F9E7818803899BB2428992B2C5
:10680000934207D39B1A9BB2081C994200D9181CCB
:1068100080B270479B1A9BB24A009B189BB2F3E769
:1068200003894089181A43425841C0B27047818891
:1068300003899BB2428992B2934206D39B1A9BB2C0
:1068400000208B424041C0B270479B1A9BB24A0065
:106850009B189BB2F4E7828803899BB2418989B275
:106860008B4206D35B1A9BB29A4208D9D01A80B2E7
:1068700070475B1A9BB251005B189BB2F4E7002093
:10688000F6E770B504000D000069002803D001216F
:10689000494202F079FC228992B263899BB22900B5
:1068A0002000FFF717FD0500618989B2A0882A0042
:1068B000FFF703FD60812069002801D002F034FC5D
:1068C000280070BD10B50023FFF712FE10BDF8B50B
:1068D00004000E00C068002803D00121494202F0E4
:1068E00053FC2589ADB22000FFF7A1FF002802D09C
:1068F000E779FF0916D0A2882B0001E09B1A9BB212
:106900009A42FBD92068E2885204520C5343C018C3
:106910003100FDF703FCA08801222900FFF7CDFC20
:1069200020810127E068002801D002F0FDFB38003B
:10693000F8BD10B50023FFF7A8FE10BD10B5040088
:10694000C068002803D00121494202F01DFC2069E3
:10695000002803D00121494202F016FC0023638184
:106960002381E068002801D002F0DEFB20690028C6
:1069700001D002F0D9FB012010BD70B504000D005C
:10698000C068002803D00121494202F0FDFB2069C4
:10699000002803D00121494202F0F6FBED01E37922
:1069A0007F2119402943E171E068002801D002F0FD
:1069B000BBFB2069002801D002F0B6FB012070BDAE
:1069C000104A53071BD0D11D0723994380239B02F4
:1069D0005B1A9B180A000C48026000214160D31822
:1069E000083B072083430948036059601960991ADE
:1069F00051601360064B1960064B19607047802385
:106A00009B02E8E7FC1B0020FC1C0220441700202E
:106A10008C1C0220801C022010B5124B1A001B682F
:106A20008342FBD351685418844208D0416844180B
:106A3000A34209D00360904200D0106010BD4068AE
:106A4000091851601000F1E7074C2468A34206D0F2
:106A50005B68C918416013681B680360EBE704605A
:106A6000E9E7C046FC1C02204417002070B5050071
:106A700001F0FEFB384B1B68002B14D0002D16D004
:106A80002B00093312D8083507231A002A402B425D
:106A900005D001339B1A093AAA4211D3ED18002DF3
:106AA00005DA00263EE0FFF78BFFE7E70025002D23
:106AB00044D02A4B1B68AB4242D3294A146803E0F6
:106AC0000025F4E722001C006368AB4202D2236871
:106AD000002BF7D1204B1B68A34233D01668083631
:106AE0002368136063685B1B102B06D9601942078B
:106AF0001ED143606560FFF78FFF626817490B681E
:106B00009B1A0B60174909688B4201D215490B602B
:106B100080231B061343636000232360124A13681B
:106B20000133136001F076FC73070DD1300070BDA6
:106B30000E4B0F4A0F48EE21FBF7A4FC0026F1E7AD
:106B40000026EFE70026EDE70B4B094A972109489D
:106B50004900FBF797FCC04644170020801C022028
:106B6000FC1C02208C1C0220981C022008A800108B
:106B700060A900103CA800107CA8001070B5002887
:106B80001ED00500083D6B68002B1ADA0200083A97
:106B90001268002A1CD1083804005B005B084360BF
:106BA00001F066FB61680E4A13685B1813602800E9
:106BB000FFF732FF0B4A13680133136001F02AFC20
:106BC00070BD094B094A42210948FF31FBF75AFCC5
:106BD000084B064AA12106484900FBF753FCC04672
:106BE000801C02209C1C0220B8A8001054A9001090
:106BF0003CA800102CA90010084B5B6A994209D8E8
:106C0000064A926A824207D2994201D0012002E0EC
:106C1000002000E0002070470120FCE70040054014
:106C200070470000000000000000000000000000AD
:106C30000B4A13681868203080F30988022080F31B
:106C40001488BFF36F8F3FBCAE4608BC04BC62B66D
:106C50001847C046C046C046C046C046C046C046AB
:106C600038170020000000000000000000000000B5
:106C7000EFF30980164B1A6820381060F0C04446C4
:106C80004D4656465F46F0C00D221207146E556EF3
:106C9000566F176F3038F0C008B572B601F08CFC33
:106CA00062B60CBC116808681030F0C8A046A9464E
:106CB000B246BB4680F309880D2212073038F0C86F
:106CC0001466556656671767F0C81847C046C04631
:106CD0003817002010B5FBF785FC000010B5002B1D
:106CE00002DB0260436010BD024B034A03483F21B0
:106CF000FBF7C8FB7097001064AA00108C97001077
:106D000010B582B00400FAF7E9FF02000B006846F4
:106D1000FFF7E4FF009A019B22606360200002B04D
:106D200010BD000030B583B004000D006846FFF7C9
:106D3000E7FF009A019B20002900801A99410A4A26
:106D400001235B4280185941002907DC02D0002052
:106D500003B030BDFA239B009842F8D3FA22920088
:106D60000023FCF771FDF3E718FCFFFF10B5031FCC
:106D7000802464041C60043B1960044B01000C393E
:106D80000B600300203B1A60403810BDD56C00102A
:106D900010B50A4B1B68002B08D1094B8022520505
:106DA0001A60BFF34F8FBFF36F8F10BD054B064ABC
:106DB00036210648FF31FBF765FBC046D01900209D
:106DC00004ED00E070A90010ECAA001090A90010DA
:106DD00072B6044A136801331360BFF34F8FBFF3D9
:106DE0006F8F7047141C0220074B1B68002B09D0C3
:106DF000064A1168BFF35F8F00221A6081F3108882
:106E0000014B1A6062B67047D0190020FC1B0220AB
:106E100010B50A4B1B68002B05D0013B074A1360D5
:106E2000002B07D010BD064B064AA7210648490093
:106E3000FBF728FBFFF7D8FFF4E7C046141C02203D
:106E4000DCA90010D8AA001090A90010EFF3108060
:106E500072B6704780F310887047000010B5FFF7D6
:106E6000F5FF040001F018FA002803D0034B80223C
:106E700052051A602000FFF7EDFF10BD04ED00E0A1
:106E800010B5094C00232360084A13600520F9F768
:106E9000CDFDFA218900FCF7B1FC0138044B1860E4
:106EA0000723236010BDC04610E000E018E000E0BA
:106EB00014E000E010B5154B1968FF2212040A43D4
:106EC0001A601968FF2212060A431A60104902204C
:106ED0004042FBF7AFFA0F4901204042FBF7AAFA04
:106EE0000D4905204042FBF7A5FAFFF7C9FF0B4B00
:106EF00000221A60D0231B061A68094B1A70FFF78C
:106F000097FE01F059FBFFF7E5FEC04620ED00E0DB
:106F1000716C00105D6E0010216C0010141C0220BA
:106F2000BD0B002010B5094B1B78D022120610684B
:106F3000834200D010BDEFF30583002B02D05B002D
:106F4000C018F7E701F080FDF4E7C046BD0B002054
:106F500000B583B0EFF30583DBB2002B10D1214BDA
:106F60001A78D0231B061B689A420FD00368BFF320
:106F70005F8F00221A6081F3108820BF03B000BD2C
:106F8000194B1A4A1A481B49FBF77CFA1A4B1B6823
:106F9000002B19D10368002B1CD0174A1360174A25
:106FA0001160174A944663449B10012199400B02DB
:106FB0001943090A134B186801235B42009300230D
:106FC000012200F019F9D9E70F4B084A08480F4988
:106FD000FBF758FA0E4B054ABA2105488900FBF722
:106FE00051FAC046BD0B0020F0A90010B4AA001051
:106FF00090A90010DB020000D0190020FC1B022029
:1070000000FFFF2F7C1C022070A90010E30200008B
:1070100050AA001030B583B00A0004681B4BE11879
:10702000891001238B4019021943090A184B1D7856
:10703000D0231B061B689D4209D040BF0368BFF3E5
:107040005F8F0021196082F3108803B030BDBFF359
:107050005F8F0023236082F31088EFF30583DBB298
:10706000002B04D10B4B186800F056F9EDE7002314
:107070000193084B186801AA00F09EF9019B002BB0
:10708000E3D0054B802252051A60DEE700FFFF2F98
:10709000BD0B00207C1C022004ED00E0F0B583B0A5
:1070A00007000E0015001C00EFF30583DBB2002B78
:1070B00030D1314B1A78D0231B061B689A422FD14E
:1070C0002E4B1B68002B38D128002100FFF72AFE29
:1070D000031E3ED03A68002A35D0284F3A6028492E
:1070E0000E6028498C4662449210012191400A02A8
:1070F0001143090A244A106800930023012200F07A
:107100007BF83B68002B2BD0204B214A2148224999
:10711000FBF7B8F9214B1E4A1E482149FBF7B2F98B
:107120000368BFF35F8F00221A6081F31088280084
:107130002100FAF75FFD040018E0144B144A1548CB
:107140001849FBF79FF9184B114A12481749FBF7EA
:1071500099F93B68BFF35F8F00221A6086F31088AD
:1071600028002100FFF748FD041E02D0200003B0D4
:10717000F0BDFFF70DFEF9E7BD0B0020D019002090
:10718000FC1B022000FFFF2F7C1C022070A90010B6
:107190007CAA001090A9001036030000F0A900108E
:1071A0001D0300002603000050AA00102E0300005B
:1071B00010B500F014F8014B186010BD7C1C0220C3
:1071C000002A03D1014206D1100003E008408842A2
:1071D00003D0002070470120FCE70120FAE710B53A
:1071E0001C20FFF743FC041E03D0002308C000F05E
:1071F000EFF8200010BD0000F0B5C64600B506004F
:107200000D001700984600282FD080235B04994278
:1072100032D2002937D001F01DFC002802D1069B94
:10722000002B37D101F024F83468424629002000B1
:10723000FFF7C6FF002834D0002F48D02300AB430F
:1072400033600023069301F0E5F8069B002B08D07D
:1072500000283FD001F030FD040083013DD5240219
:10726000240A200080BCB846F0BD254B254A3C21AD
:107270002548FF31FBF706F9244B224A9E2122487C
:107280004900FBF7FFF8224B1E4A3E211E48FF3102
:10729000FBF7F8F81F4B1B4AA0211B484900FBF7DE
:1072A000F1F8069B002BCED0002F0DD100214346D4
:1072B000002B02D08023DB0419432943301D069A9A
:1072C00001F0ECF90024BEE780214904EFE7002338
:1072D0000693B8E7FFF75CFDBCE7FFF779FD34687C
:1072E000424629002000FFF76BFF002804D0002F42
:1072F00002D02300AB433360FFF78AFDAFE7C046FF
:10730000F8AA001008AC001004AB00103CAB001051
:1073100064AB00107CAB0010F8B504000D00002831
:107320000DD080235B0499420FD206000C3600F08A
:107330009FFF206923682B432360002718E0174B29
:10734000174A18481849FBF79DF8184B144A85212D
:1073500014488900FBF796F821681940994206D134
:1073600011E0236880218904194301F087FA28007D
:10737000B0420CD04568026813021B0A5101EBD4DD
:1073800021680B42F3D0D201EBD51F43E9E7236814
:10739000BB43236001F03EF82068F8BDF8AA001056
:1073A000F4AB001004AB001013020000D0AB0010CF
:1073B00010B5FFF7B1FF10BD10B51300034C0A0064
:1073C0000100200001F048FE10BDC046B17300105E
:1073D000030008334360012252428260C3600361AC
:1073E00000230360704700230361704730B50D68C8
:1073F0006B1C10D0030008331C005B681A68AA429B
:10740000FAD963684B6099608C60616008610368B9
:107410000133036030BD0469F3E7036941688268A2
:107420008A60416851605A68824206D00022026137
:107430001A68013A1A601868704782685A60F5E75E
:107440000300406A002803D01B6B1B682020C01A71
:10745000704710B50400FFF7BBFCA26BE36B9A42C8
:1074600004D00024FFF7D4FC200010BD0124F9E76C
:1074700010B50400FFF7ACFCA36B002B04D1012472
:10748000FFF7C6FC200010BD0024F9E770B504002A
:107490001500866B026C002A0CD10368002B03D008
:1074A00000200136A66370BD806801F03FFB002319
:1074B000A360F6E7002D0DD14068FCF72FFE63684E
:1074C000226C9B186360A26893421AD3236863609E
:1074D0002800E6E7C068FCF721FEE368226C514211
:1074E0009B1AE3602268934202D2A3685B18E360B0
:1074F000022D01D00020D4E7002E04D0013E002050
:10750000CFE72800CDE70020CBE710B50300080047
:107510001A6C002A0AD0DC68A418DC6099688C42D6
:1075200001D31968D960D968FCF7F8FD10BD0000D7
:1075300070B582B00190846C002C0AD0A26BE36B12
:107540009A420DD2A26B934210D80025280002B0B7
:1075500070BD1A4B1A4AC2211A480901FAF792FF64
:10756000194B174A17481949FAF78CFF4523E65C6F
:1075700076B2002201A92000FFF788FF0500731CE6
:107580000AD1636A002BE1D02000243001F0F6F824
:107590000028DBD00125D9E700F078FE8642D5D25D
:1075A0007F2E04D0013676B24523E654CEE7084B51
:1075B000034A04480749FAF765FFC0461CAC0010AF
:1075C000F0AE001030AC001060AC0010210C0000D8
:1075D000A8AC0010410C000070B50500FFF7F8FBE7
:1075E0004523EC5C64B20AE06B6A002B17D02800DC
:1075F000243001F0C3F800280ED1013C64B2002C05
:107600000DDDAB6C002BEFD02800FFF791FF0028B9
:10761000F3D001F013FAF0E701F010FAEDE745239B
:10762000FF22EA54FFF7F4FBFFF7D2FB4423EC5CA4
:1076300064B201E0013C64B2002C0BDD2B69002B2D
:1076400008D02800103001F099F80028F2D001F09D
:10765000F5F9EFE74423FF22EA54FFF7D9FB70BDA9
:10766000F8B504000D0000282BD0C36B002B54D0BC
:10767000026C0026190C100C002937D181B20029A8
:1076800026D1002E49D1FFF7A3FB2268E36B206CC3
:10769000010059435118A1600021A1636260013BC0
:1076A0004343D218E260FF234422A3540132A3547F
:1076B000002D29D12369002B1DD1FFF7A9FB012043
:1076C000F8BD194B194A972119484900FAF7DAFE13
:1076D000011C181C9BB292B25A4380B289B241433A
:1076E000120C8918090CCCD00126CAE780B20028F8
:1076F000FAD1101CEEE72000103001F03FF800280E
:10770000DBD0FFF745FBD8E720001030FFF760FE25
:1077100020002430FFF75CFECFE7064B034A6421CC
:107720000348FF31FAF7AEFECCAC001034AF0010C6
:1077300030AC0010D4AC001070B51D00049C0029C2
:107740000BD12460E063216401212000FFF788FF52
:107750005023E5540023A36470BD2260F2E70000CB
:10776000F0B583B004000F001600002831D00021CE
:10777000030C3A0C002B27D193B2002B16D1002911
:1077800027D1380060430300553322D85430FFF727
:107790006DF9051E07D00200543200903300390005
:1077A0002000FFF7C9FF280003B0F0BD131C201C08
:1077B000A5B2BAB26A4380B29BB24343120C9B1883
:1077C0001B0CDCD00121DAE792B2002AFAD1381C76
:1077D000EEE7034B034A04480449FAF753FEC04658
:1077E000F8AC001020AF001030AC00101502000003
:1077F000F0B585B004000F0001921E00002813D0E0
:10780000002917D0022E02D1E36B012B1BD101F00E
:1078100021F9051E1DD1019B002B5BD04D4B4E4A1B
:107820004E484F49FAF72EFE4E4B4B4A4B484E49B5
:10783000FAF728FE036C002BE4D04C4B464A47482D
:107840004B49FAF71FFE4B4B434A44484A49FAF763
:1078500019FE00253EE0A56B320039002000FFF73D
:1078600015FEA36C002B10D0022E01D1002D04D1E7
:107870002000FFF75DFE002804D1FFF7C9FA0120C0
:1078800005B0F0BDFFF784FAF7E7636A002B04D177
:107890000028F2D0FFF77CFAEFE72000243000F058
:1078A0006DFF0028E9D0FFF773FAE6E7FFF7B0FABB
:1078B0000020E5E702A801F05BF8013517E000229F
:1078C000E2541FE00022E25421E02000FFF784FE92
:1078D00000F0A0FDFFF77CFAA26BE36B9A42BAD3EB
:1078E000022EB8D0019B002BE0D0002DE2D0FFF794
:1078F0008FFA00F0BDFCFFF76BFA4423E25C52B252
:107900000132DCD04523E25C52B20132DAD0FFF71B
:107910007FFA01A902A801F037F8002813D120004E
:10792000FFF797FD0028D0D001992000103000F01B
:1079300097FE2000FFF750FE00F06CFD0028C9D133
:10794000FFF726FAC6E72000FFF746FE00F062FDCB
:10795000002095E77CAB00100CAF001030AC00109D
:1079600082030000CCAC00107D03000004AD0010C9
:107970007E0300005CAD00107F03000010B50028FE
:1079800007D0002383600360C36000220021FFF75B
:107990002FFF10BD10B5020000210120FFF7E0FE0F
:1079A0000400FFF7EBFF200010BD0000F0B5D64645
:1079B000474680B583B004000F0001921D000028E7
:1079C00019D000291DD0022D02D1E36B012B21D14A
:1079D000FFF73CFA8046A26BE36B9A4220D3022D5C
:1079E0001ED000244046FFF735FA200003B0C0BC8B
:1079F000BA46B046F0BD324B324A33483349FAF703
:107A000041FD036C002BDED0314B2E4A2E4831490C
:107A1000FAF738FD304B2B4A2B483049FAF732FD44
:107A20004523E65C76B2A36B9A462A003900200013
:107A3000FFF72CFD731C25D1A36C002B10D0022D59
:107A400002D15346002B2FD12000FFF771FD0028F3
:107A50002CD0019A002A2BD0012313600124C1E706
:107A6000636A002B01D10124BCE72000243000F020
:107A700085FE00281ED0019A002A1DD00123136024
:107A80000124AFE700F002FC864217D27F2E05D01A
:107A9000013676B24523E6540124A3E7104B094A88
:107AA00009481049FAF7EEFC01249BE7012499E705
:107AB000012497E7012495E7012493E7012491E746
:107AC000CCAC0010D4AE001030AC0010510400005B
:107AD00004AD0010520400005CAD0010530400001F
:107AE000A8AC0010DC040000F0B585B004000E0066
:107AF000019200280ED0002912D000F0ABFF051E25
:107B000018D1019B002B4FD0434B444A4448454970
:107B1000FAF7B8FC444B414A41484449FAF7B2FCF1
:107B2000036C002BE9D0424B3C4AB4213C48C900CD
:107B3000FAF7A8FC002537E031002000FFF7E5FC4C
:107B4000013FA7632369002B04D1FFF761F90120EE
:107B500005B0F0BD2000103000F010FE0028F4D079
:107B6000FFF716F9F1E7FFF753F90020F0E702A855
:107B700000F0FEFE013521E044230022E25428E01B
:107B800045230022E25429E02000FFF725FD00F004
:107B900041FC09E02000FFF71FFD00F03BFC200046
:107BA000FFF766FC002835D1FFF712F9A76B002F0D
:107BB000C2D1019B002BD6D0002DD8D0FFF728F9D9
:107BC00000F056FBFFF704F94423E35C5BB201339A
:107BD000D2D04523E35C5BB20133D1D0FFF718F973
:107BE00001A902A800F0D0FE0028D3D12000FFF7A1
:107BF0003FFC0028C8D001992000243000F030FD5F
:107C00002000FFF7E9FC00F005FC0028CCD1FFF7CD
:107C1000BFF8C9E700209BE77CAB0010C4AE0010A2
:107C200030AC0010A50500002CAE00109C05000033
:107C300038AE001070B584B0041E01910BD0036CF7
:107C4000002B0ED100F006FF061E16D1019B002B63
:107C50000DD1050058E0514B514A52485249FAF7AC
:107C600011FC524B4E4A4F485149FAF70BFC514B0D
:107C70004B4A4C485049FAF705FC0025002643E0E2
:107C8000013BA3632368002B07D02369002B08D195
:107C9000FFF7BEF8012004B070BD01F019F8A06034
:107CA000F3E72000103000F069FD0028F0D0FFF766
:107CB0006FF8EDE7FFF7ACF80020ECE702A800F062
:107CC00057FE01362AE044230022E25431E04523E6
:107CD0000022E25432E0FFF77BF8A06800F0CCFE0F
:107CE0000500FFF795F839E02000FFF775FC00F07C
:107CF00091FB09E02000FFF76FFC00F08BFB2000F8
:107D0000FFF7B6FB002838D1FFF762F8A36B002B12
:107D1000B6D1019B002BCDD0002ECFD0FFF778F845
:107D200000F0A6FAFFF754F84423E35C5BB201339A
:107D3000C9D04523E35C5BB20133C8D0FFF768F8D4
:107D400001A902A800F020FE0028D3D12000FFF7EF
:107D50008FFB0028C8D02368002BBCD001992000DD
:107D6000243000F07DFC2000FFF736FC00F052FBD1
:107D70000028C9D1FFF70CF8C6E7002D01D100207B
:107D800089E7FFF725F82000FFF75AFB0100A068FC
:107D900000F02CFFFFF73CF8F1E7C0462CAE0010D6
:107DA000B0AE001030AC00102E060000ACAD0010DC
:107DB000320600007CAB00103706000070B50028CA
:107DC00004D0002922D00024002209E0104B114ADF
:107DD00011481249FAF756FB114BEC1814E0013226
:107DE000072A0FD80E4BD5005B195B688342F3D08E
:107DF000002CF4D10A4BD500EB58002BEFD1084BE7
:107E0000EC18ECE7002C01D02160606070BDC0462A
:107E100094AE00109CAE001030AC0010150B0000AA
:107E2000B81C022070B504000D001600FEF7D0FF4C
:107E30004423E35C5BB201330DD04523E35C5BB2CA
:107E400001330CD0FEF7E4FFA36B002B0BD0200016
:107E5000FFF7C2FB70BD44230022E254EDE7452347
:107E60000022E254EEE7200024303200290000F026
:107E700055FCECE7084B1B681B68002B04D1074B33
:107E8000012252421A607047034B1B68DB681A6874
:107E9000024B1A60F7E7C04640170020901C0220F2
:107EA00010B50400006BFEF769FE2000FEF766FEC9
:107EB00010BD0000F0B5DE4657464646C0B58246C6
:107EC0000F0014009B46089E0A9D286B9200A52176
:107ED000FCF71EF92B6B1E4A94466444A4001B1940
:107EE000072293439846002F0DD000240F2C07D86B
:107EF0003A5D2B1934331A70002A01D00134F5E7AA
:107F000043230022EA541F2E1CD8EE62EE64281D83
:107F1000FFF769FA28001830FFF765FA2D61202372
:107F20009B1BAB616D625A4651464046FEF71EFFF1
:107F30002860099B002B00D01D60E0BCBB46B24608
:107F4000A846F0BD034B044A04480549FAF79AFADB
:107F5000FFFFFF3F80AF001050B2001050AF001085
:107F60009603000070B5002407E0A3001B199800D9
:107F70000E4BC018FFF72CFA01341F2CF5D90C4D0D
:107F80002800FFF725FA0B4C2000FFF721FA0A48DA
:107F9000FFF71EFA0948FFF71BFA0948FFF718FA1E
:107FA000084B1D60084B1C6070BDC0465017002078
:107FB000541C0220681C0220A41C0220181D022050
:107FC000041D0220401700204817002010B50400AF
:107FD000FEF7FEFE284A136801331360274B1B6827
:107FE000002B0CD0264B1B68002B0DD1234B1B689C
:107FF000DA6AE36A9A4207D8204B1C6004E01F4B00
:108000001C601368012B31D01E4A136801331360C2
:108010006364E16A1C4B1B68994201D91A4B1960D1
:108020001A4A8B005B189B00D3185B68A3609868A2
:10803000E060211D41609960E06A830019188900A1
:108040008918616119188900895801311B189B0032
:108050009950FEF7DDFE0A4B1B68002B05D0074B3D
:108060001B68DA6AE36A9A4203D310BDFFF77AFF0E
:10807000CAE7FEF78DFEF8E7181C0220381700202B
:10808000F81C0220241C0220281C0220501700206B
:1080900010B514E0FEF79CFE0B4BDB68DC68201D7E
:1080A000FFF7BBF9094A1368013B1360084A1368DC
:1080B000013B1360FEF7ACFE2000FFF7F1FE044B1E
:1080C0001B68002BE6D110BD181D0220181C0220D1
:1080D0001C1C022010B5FFF7DBFF034B1B68012BB4
:1080E000F9D9FEF755FEF6E75017002070B50400E9
:1080F0000D001F4B1E681F4B19686D22002088540D
:1081000018680430FFF789F9631C0DD03419194B36
:108110001B685C60A6421DD9174B1868154B19687F
:108120000431FFF763F970BD002DEFD0134A516899
:10813000104B1868816018688C68C4601868043037
:1081400060601868043088601B685A6113680133E6
:108150001360E8E70A4B1868064B19680431FFF70B
:1081600045F9084B1B68A342DDD9064B1C60DAE7D2
:108170002C1D02203817002048170020041D022063
:1081800040170020901C0220F0B587B004900591A4
:1081900016001F009000FEF769FC041E21D070201D
:1081A000FEF764FC051E16D070220021FBF7B0FF1D
:1081B0002C630023039302950D9B01930C9B00936A
:1081C0003B00320005990498FFF774FE2800FFF782
:1081D000FDFE012007E02000FEF7D0FC0120404218
:1081E00001E00120404207B0F0BD000000B583B0BF
:1081F000802215491548164B019300230093520025
:10820000FFF7C2FF012805D0013015D0114B1B68C4
:1082100003B000BD00F0F4FE0128F5D172B60E4B9C
:10822000012252421A600D4B02321A600C4B00229E
:108230001A60FEF73FFEE9E70A4B0B4A82210B4822
:108240000901FAF71FF9C046BCAF0010D580001035
:10825000841C0220C00B0020901C0220F81C02206D
:108260002C1D0220C4AF001030B2001050AF00101F
:10827000024A1368013313607047C046201C022075
:10828000014B18687047C0462C1D0220014B18682E
:108290007047C046181C0220F8B54F4B1B68002BD6
:1082A00000D093E04D4B1E6801361E60002E10D1A9
:1082B0004B4B1B681B68002B21D1494A1168494B65
:1082C000186810601960484A136801331360FFF79B
:1082D000D1FD464B1B68B34217D90020444B1B68A5
:1082E000D96A444A8B005B1899008B58012B00D93E
:1082F0000120414B1B68002B6DD001206BE03F4BF0
:108300003F4A40484049FAF7BDF8002033E0374B78
:10831000012252421A60E1E7344B1A60DEE7D96865
:1083200051603EE000219962116801391160DA6AFA
:10833000364909688A4201D934490A602D499400B6
:10834000A418A2008A1852689A609468DC6065607C
:108350009560DC6AA2001719BD006D185D61BD0053
:108360006D580135BC006550DA6A214B1B68DB6A29
:108370009A4200D901201A4B1B681B68002BC6D0FB
:10838000174B1B68DB68DB685A689642C4D35A698E
:108390009C68D968A1609C684C6051681D1DA94209
:1083A000BDD0002159611168013911609A6A002A13
:1083B000BDD0DC69196AA160DC694C6054681900A1
:1083C00018318C42AED1196A5160ABE7104A13687C
:1083D000013313600020F8BD201C02202C1D022058
:1083E0004017002048170020941C0220901C0220F7
:1083F0003817002050170020381D0220D8AF001079
:108400000CB2001050AF0010F40A0000281C02202B
:10841000A01C022010B54A4B1B68002B0FD0FEF7A2
:10842000D7FC474B1A68013A1A601B68002B00D032
:1084300080E0444B1B68002B0DD100247BE0424BB5
:10844000424A43484349FAF71DF8196A516015E05A
:10845000D968516021E000233F4A1268002A4AD0BF
:108460003D4BDB68DB689A6AD869196A8160D86914
:1084700048605068190018318842E6D0002199629E
:108480001168013911605A699868D96881609868E3
:10849000486051681C1DA142DAD000215961116861
:1084A00001391160D86A2D4A1268904201D92B4ACD
:1084B00010602B498200121892008A1852689A6044
:1084C0009068D86044609460DC6AA2001019800053
:1084D000401858611019800040580130121992005C
:1084E0005050D96A1F4A1268D26A9142B4D91E4AC2
:1084F00001211160B0E7002B01D0FFF7BBFC1B4B43
:108500001C68002C0AD1184B1C68002C13D0FEF7F5
:108510003FFC01240FE0013C002C07D0FFF7BCFE1C
:108520000028F8D0104B01221A60F4E70F4B00220C
:108530001A60E8E70024FEF76BFC200010BDC0467F
:10854000201C0220181C022050B0001020B2001085
:1085500050AF001093080000A41C0220281C022029
:108560005017002038170020381D0220A01C0220C0
:1085700010B5041E0DD00C4B1B68002B0CD1FFF75F
:1085800077FE00212000FFF7B1FDFFF743FF002831
:1085900001D1FEF7FDFB10BD044B054AA42105489F
:1085A000C900F9F76FFFC046201C022090AF0010F1
:1085B00044B2001050AF001010B5204B1B68002BC8
:1085C00003D01F4B01221A6010BD1D4B00221A6000
:1085D0001C4B1B681C499A00D21890004258002A74
:1085E00009D1002B01D0013BF4E7184B184A194878
:1085F0001949F9F747FF08009900CC18A200821822
:10860000546864685460C9188A0008321218944289
:108610000BD00D4A9900C918880012185268D16809
:108620000E4A1160074A1360CEE702009900C9188C
:1086300088001218D1685160EBE7C046201C022068
:10864000381D0220281C0220501700207CB000108A
:10865000F8B1001050AF0010330C000038170020A4
:1086600010B50C00002809D0074B19681831FEF727
:10867000BDFE01212000FFF739FD10BD034B044A68
:1086800004480549F9F7FEFE381700208CB00010A9
:10869000E0B1001050AF00104B0C000070B50300AB
:1086A0001000002B1ED0154A1268002A20D0144C4E
:1086B0002568802212060A43AA615A682168CA61A5
:1086C000216895680D622168183169602168183148
:1086D0009160226893621A6801321A600121FFF7E3
:1086E00005FD70BD074B084A08480949F9F7CAFE5D
:1086F000084B054A05480849F9F7C4FE201C02202A
:10870000381700208CB00010C0B1001050AF00101E
:10871000650C000050B00010690C000070B503003B
:1087200008001100002B18D05A680F4C2568EA6128
:10873000256896682E622568183575602568183595
:108740009560226893621A6801321A60002901D08C
:1087500001204042FFF7CAFC70BD044B044A0548A3
:108760000549F9F78FFEC046381700208CB000107D
:10877000A0B1001050AF0010810C000010B5C3680C
:10878000DB68002B4CD09A6AD869196A8160D86975
:108790004860516818001830814247D00021996222
:1087A0001168013911602B4A1268002A44D15A69B4
:1087B0009868D96881609868486051681C1DA1421A
:1087C00037D000215961116801391160D86A224AF5
:1087D0001268904201D9204A106020498200121884
:1087E00092008A1852689A609068D86044609460D9
:1087F000DC6AA2001019800040185861101980002E
:1088000040580130121992005050DA6A144B1B681C
:10881000DB6A9A421CD9134B01221A60012018E02E
:10882000114B124A12481349F9F72CFE196A51608C
:10883000B4E7D9685160C4E70F4A5168D9618C68C0
:108840001C62606088609A62116801311160DCE727
:10885000002010BD201C0220281C022050170020E0
:1088600038170020381D022098B0001084B1001085
:1088700050AF0010B10C0000A41C022010B5314B09
:108880001B68002B4CD080231B060B430360C3687E
:10889000002B4BD0026944688168A16044684C6039
:1088A0005168814248D0002101611168013911608D
:1088B0005A699868D96881609868486051681C1D39
:1088C000A1423CD000215961116801391160D86A78
:1088D0001D4A1268904201D91B4A10601B49820050
:1088E000121892008A1852689A609068D8604460A2
:1088F0009460DC6AA20010198000401858611019B9
:10890000800040580130121992005050DA6A104B22
:108910001B68DB6A9A4202D90E4B01221A6010BD15
:108920000D4B0E4A0E480F49F9F7ACFD0E4B0B4AA2
:108930000B480E49F9F7A6FD81685160B3E7D96885
:108940005160BFE7201C0220281C02205017002085
:1089500038170020381D022050B0001060B1001000
:1089600050AF0010E90C000098B00010F10C0000AE
:10897000034B1B680360034B1B6843607047C04692
:10898000941C02202C1D0220F8B504000D000028C4
:1089900017D000291BD0FEF71BFA1F4B1A6863681B
:1089A000D61A1E4908686D21415C002915D01B4B61
:1089B0001A686D230021D1540124FEF729FA200002
:1089C000F8BD174B174A18481849F9F75BFD184BC3
:1089D000144A15481749F9F755FD2968481C18D05D
:1089E000276815480068874205D0934203D80023C2
:1089F0002B600124E1E7B14203D800232B6001245E
:108A0000DBE79B1A5B182B602000FFF7B1FF002407
:108A1000D3E70024D1E7C0462C1D022038170020E0
:108A2000A8B0001048B1001050AF00102C0D00008D
:108A3000B4B000102D0D0000941C0220014B012247
:108A40001A607047381D0220014B18687047C046F5
:108A500038170020064B1B68002B07D0054B1B68FE
:108A6000002B01D0002002E0022000E0012070472E
:108A7000F81C0220201C022070B5041E4CD0C26AD3
:108A8000274B1B68DB6A9A423ED28369002B05DBC9
:108A9000234B1B68D96A20235B1A836161699300A9
:108AA0009B189B001F4A9B18994205D01C4B1B68C2
:108AB000DB6AE362012030E0251D2800FEF7ADFCF3
:108AC000174B1B68D96AE162174B1B68994201D9A1
:108AD000154B1960134A8B005B189B00D3185B6819
:108AE000A3609968E1604D609D60E06A8300191899
:108AF00089008918616119188900895801311B188A
:108B00009B009950012008E0C26C054B1B68DB6A92
:108B10009A4203D3002000E0002070BD0120FCE752
:108B20003817002050170020281C022070B5041EA2
:108B300045D0254B1B6883420CD1036D002B0FD011
:108B4000013B0365C16AC26C91423AD0002B0DD043
:108B5000002070BD1D4B1E4A1E481F49F9F792FCAC
:108B60001E4B1B4A1B481E49F9F78CFC051D2800AB
:108B7000FEF753FCE16CE16220235B1AA361194B01
:108B80001B68994201D9174B1960174A8B005B1873
:108B90009B00D3185B68A3609968E1604D609D609D
:108BA000E06A830019188900891861611918890021
:108BB000895801311B189B0099500120C9E70020FA
:108BC000C7E70020C5E7C04638170020C4B0001032
:108BD00030B1001050AF00108C100000DCB000105D
:108BE0008D100000281C02205017002070B5041EB4
:108BF0000BD0026D002A09D0C36C8B4200D20B004F
:108C0000E16A994201D0012A06D070BD214B224A67
:108C100022482349F9F736FC224A1268A24232D090
:108C2000E362A269002A02DB2022D31AA3616269EF
:108C30008B005B189B001C495B189A42E5D1251DEF
:108C40002800FEF7EAFBE16A184B1B68994201D93C
:108C5000164B1960144A8B005B189B00D3185B6895
:108C6000A3609968E1604D609D60E06A8300191817
:108C700089008918616119188900895801311B1808
:108C80009B009950C1E70A4B034A04480949F9F788
:108C9000F9FBC046DCB000100CB1001050AF001062
:108CA000DC1000003817002050170020281C02207C
:108CB000F4B00010F7100000044B1A6890691A68AD
:108CC000D16A1A6820235B1A936170473817002015
:108CD000054B1B68002B04D0034B1A68136D01333E
:108CE0001365014B1868704738170020074B1A6846
:108CF0001368002B06D101330360002B04D1D36825
:108D0000186870470023F7E70020FAE73C170020B7
:108D100010B54160006191420CD8D21A83699A4221
:108D200001D3012010BD011D094B1868FEF75EFB41
:108D30000020F7E79A4201D2994206D2011D054B65
:108D40001868FEF753FB0020ECE70120EAE7C04675
:108D50004C1700203C17002070B504000D001600D1
:108D600004E0A369ED18236A20009847A169491916
:108D70002B0032002000FFF7CBFF0028F1D170BD9F
:108D800070B505000E000C4B1B68DB68DC68201D0D
:108D9000FEF743FB2823E35C5A0707D401229343E1
:108DA0002732A354236A2000984770BD320029005F
:108DB0002000FFF7D1FFF5E73C17002010B505E0D4
:108DC000DB68186801214942FFF7DAFF054B1B6891
:108DD0001A68002AF4D1034A0349086810600B603E
:108DE00010BDC0463C1700204C17002070B5050090
:108DF000FFF746FA0400074B1B68834205D800239F
:108E00002B60044B1C60200070BDFFF7D7FF0123CF
:108E10002B60F6E7881C022070B582B004000D00BC
:108E2000FFF726FA01A8FFF7E1FF0600019B002BE0
:108E300022D1002D14D1A0420BD2A11B104B1868D7
:108E40002A00FEF7EFFFFFF7E5FA002811D002B085
:108E500070BDFFF7DFFA31002000FFF791FFF6E762
:108E6000084A12681268002A01D10125E5E71D00B1
:108E7000E3E7FDF78DFFEAE7FFF7CCFAE7E7C04647
:108E8000301D02204C17002030B587B002E0029B55
:108E9000002B0FDA374B1868002202A9FEF724FED8
:108EA000002865D0029B002BF1DA039B04980599FA
:108EB0009847ECE7049C6369002B02D0201DFEF765
:108EC000ACFA01A8FFF792FF050002990929E1D841
:108ED0008900294B59588F462822A35C01210B4356
:108EE000A354039BA169591802002000FFF710FF4B
:108EF0000028CFD02823E35C5A0707D401229343EC
:108F00002732A354236A20009847C3E70399A36933
:108F1000C9182A002000FFF71FFFF3E72822A35CEF
:108F200001218B43A354B5E72822A35C01210B4305
:108F3000A3540399A161002906D009180300020077
:108F40002000FFF7E5FEA5E70C4B0D4ADD310D488B
:108F50008900F9F797FA2823E35C9A0704D50122E0
:108F600093432732A35495E72000FDF707FE91E7CE
:108F700007B030BD301D0220C0B2001068B2001032
:108F800000B3001090B2001000B583B001A8FFF745
:108F9000ADFE0199FFF740FFFFF776FFF6E700000F
:108FA00070B5FDF715FF104B1B68002B02D0FDF7C5
:108FB0002FFF70BD0D4D2800FEF70AFA0C4C200063
:108FC000FEF706FA0B4B1D600B4B1C6000221021B4
:108FD0000A20FEF7C5FB044B18600028E7D00749BC
:108FE000FEF7ECFEE3E7C046301D02202C1C0220F9
:108FF000401C02203C1700204C170020E8B2001053
:1090000000B583B0FFF7CCFF0C4B1B68002B0ED0D4
:1090100080220B490B480C4B01931F230093002324
:10902000D200FFF7B1F8002801D003B000BD074B14
:10903000074A1A210748FF31F9F724FA301D0220A8
:10904000F0B20010898F0010341D0220F8B2001019
:109050001CB3001090B2001010B584B014001A00B8
:1090600002235B420093019002910394034B186822
:1090700000236946FEF79AFC04B010BD301D0220A3
:109080000123084A1360084A1360084B9A680123B9
:109090009343FAD1064B01221A60054B1B68DB058E
:1090A000FBD5704700E0004000F0004000C00040E9
:1090B00000C0044010B583070AD00300032102E07A
:1090C00001330B4205D01A78002AF9D1181A10BDC5
:1090D000030019680C4A0D4C8A188A4322420FD1AA
:1090E0005968094A04338A188A43224208D15968C8
:1090F000054A04338A188A432242F1D000E0013342
:109100001A78002AFBD1E1E7FFFEFEFE8080808016
:10911000F8B5C0460000000001B40248844601BC16
:10912000604700BF2501002001B40248844601BC0D
:10913000604700BFFD02002001B40248844601BC24
:10914000604700BF210A002001B40248844601BCE8
:10915000604700BF3D03002001B40248844601BCC3
:10916000604700BF0506002001B40248844601BCE8
:10917000604700BF210A002001B40248844601BCB8
:10918000604700BFFD01002001B40248844601BCD5
:10919000604700BFE302002001B40248844601BCDE
:1091A000604700BF7508002001B40248844601BC36
:1091B000604700BFD905002001B40248844601BCC5
:1091C000604700BFB102002001B40248844601BCE0
:1091D000604700BFA907002001B40248844601BCD3
:1091E000604700BF4507002001B40248844601BC27
:0891F000604700BF5107002099
:1091F8006C65667420776865656C3A2025640A009A
:10920800726967687420776865656C3A20256620FE
:10921800726F756E64730A006D6F6E69746F725F3A
:109228006C6566745F776865656C5F7370656564A7
:109238005F7461736B0000006D6F6E69746F725FAD
:1092480072696768745F776865656C5F7370656578
:10925800645F7461736B00006C656E203E203000A3
:109268002F55736572732F72712F7069636F2F702A
:1092780069636F2D73646B2F7372632F7270325F23
:10928800636F6D6D6F6E2F7069636F5F756E697157
:1092980075655F69642F756E697175655F69642EA0
:1092A800630000007069636F5F6765745F756E695E
:1092B8007175655F626F6172645F69645F73747210
:1092C800696E6700666C6173685F6F666673202BF2
:1092D80020636F756E74203C3D205049434F5F46B4
:1092E8004C4153485F53495A455F425954455300CE
:1092F8002F55736572732F72712F7069636F2F709A
:1093080069636F2D73646B2F7372632F7270325F92
:10931800636F6D6D6F6E2F68617264776172655FE0
:10932800666C6173682F666C6173682E6300000059
:10933800636F6E6E6563745F696E7465726E616C7F
:109348005F666C61736820262620666C6173685FAF
:10935800657869745F78697020262620666C617369
:10936800685F72616E67655F657261736520262646
:1093780020666C6173685F666C7573685F636163B0
:1093880068650000636F6E6E6563745F696E74650F
:10939800726E616C5F666C61736820262620666C4D
:1093A8006173685F657869745F7869702026262024
:1093B800666C6173685F72616E67655F70726F6714
:1093C80072616D20262620666C6173685F666C7515
:1093D80073685F636163686500000000636F6E6EA9
:1093E8006563745F696E7465726E616C5F666C61EB
:1093F800736820262620666C6173685F65786974D7
:109408005F78697020262620666C6173685F666CD9
:109418007573685F6361636865000000666C6173FB
:10942800685F646F5F636D64000000004E6F2073B7
:1094380070696E6C6F636B73206172652061766111
:10944800696C61626C6500007372635F6672657156
:10945800203E3D2066726571000000002F5573653F
:1094680072732F72712F7069636F2F7069636F2D1C
:1094780073646B2F7372632F7270325F636F6D6DDD
:109488006F6E2F68617264776172655F636C6F637A
:109498006B732F636C6F636B732E6300636C6F6306
:1094A8006B5F636F6E6669677572650030783163EC
:1094B800203D3D20282A696E7374293E3E3131755E
:1094C800000000002F55736572732F72712F706939
:1094D800636F2F7069636F2D73646B2F7372632FC3
:1094E8007270325F636F6D6D6F6E2F686172647733
:1094F8006172655F6972712F6972712E6300000075
:1095080064656C7461203E3D202D3230343820264D
:10951800262064656C7461203C3D2032303436204E
:10952800262620212864656C7461202620312900B4
:10953800212864656C7461203E3E20313175290014
:1095480063757272656E74203D3D205F5F756E684D
:10955800616E646C65645F757365725F69727120B2
:109568007C7C2063757272656E74203D3D20686155
:109578006E646C65720000006972715F68616E6488
:1095880065725F636861696E5F667265655F736C5B
:109598006F745F68656164203E3D20300000000004
:1095A800767461626C655F68616E646C6572203D9B
:1095B8003D205F5F756E68616E646C65645F75738E
:1095C80065725F6972710000212828282875696E04
:1095D800747074725F7429767461626C655F686117
:1095E8006E646C657229202D20282875696E747048
:1095F80074725F74296972715F68616E646C6572F8
:109608005F636861696E5F736C6F747329202D20C6
:1096180031292573697A656F662873747275637466
:10962800206972715F68616E646C65725F636861FE
:10963800696E5F736C6F7429290000002165786377
:10964800657074696F6E207C7C20657863657074C2
:10965800696F6E203D3D206E756D202B205654415C
:10966800424C455F46495253545F495251000000ED
:1096780066616C736500000069735F736861726589
:10968800645F6972715F7261775F68616E646C654F
:109698007228736C6F745F68616E646C6572290000
:1096A800657863657074696F6E000000666F756E2B
:1096B800640000004E6F2075736572204952517323
:1096C8002061726520617661696C61626C65000079
:1096D8006972715F6164645F7461696C5F746F5F04
:1096E800667265655F6C697374000000696E736506
:1096F80072745F6272616E63685F616E645F6C69E9
:109708006E6B00006972715F72656D6F76655F6878
:10971800616E646C657200006D616B655F62726199
:109728006E6368007265736F6C76655F6272616EF6
:10973800636800006972715F6164645F7368617275
:1097480065645F68616E646C657200006972715F60
:109758007365745F6578636C75736976655F686156
:109768006E646C657200000075735F73696E636583
:109778005F626F6F74203C3D20494E5436345F4D14
:10978800415800002F55736572732F72712F7069DD
:10979800636F2F7069636F2D73646B2F7372632F00
:1097A800636F6D6D6F6E2F7069636F5F6261736554
:1097B8002F696E636C7564652F7069636F2F747998
:1097C8007065732E68000000746F74616C0000008F
:1097D8002F55736572732F72712F7069636F2F70B5
:1097E80069636F2D73646B2F7372632F636F6D6D75
:1097F8006F6E2F7069636F5F73796E632F6D757409
:1098080065782E63000000006D74782D3E636F72DA
:10981800652E7370696E5F6C6F636B006C6F636B42
:109828005F69735F6F776E65725F69645F76616C9D
:109838006964286D74782D3E6F776E657229000013
:109848006D74782D3E656E7465725F636F756E74A6
:10985800000000006D757465785F657869740000B4
:109868006D757465785F656E7465725F626C6F6341
:109878006B5F756E74696C007570646174655F7593
:10988800735F73696E63655F626F6F7400000000D9
:109898006964202626206964203C3D20706F6F6C27
:1098A8002D3E686561702D3E6D61785F6E6F6465F1
:1098B800730000002F55736572732F72712F7069D2
:1098C800636F2F7069636F2D73646B2F7372632FCF
:1098D800636F6D6D6F6E2F7069636F5F74696D650F
:1098E8002F74696D652E63006964202626206964DB
:1098F800203C3D20686561702D3E6D61785F6E6F1C
:10990800646573002F55736572732F72712F7069B8
:10991800636F2F7069636F2D73646B2F7372632F7E
:10992800636F6D6D6F6E2F7069636F5F7574696CAF
:109938002F696E636C7564652F7069636F2F75741A
:10994800696C2F70686561702E68000070617265BF
:109958006E745F69640000006368696C645F6964C1
:1099680000000000706172656E745F696420213DBB
:10997800206368696C645F696400000069640000C2
:109988006964202626202170685F636F6E746169A0
:109998006E735F6E6F646528686561702C206964FA
:1099A8002900000021686561702D3E667265655F5B
:1099B8007461696C5F6964002170685F636F6E74BD
:1099C80061696E735F6E6F646528706F6F6C2D3E92
:1099D800686561702C2072657573655F696429001C
:1099E80072656D6F7665645F6964203D3D206E65C4
:1099F80078745F696400000063616C6C6261636B1A
:109A080000000000706F6F6C2D3E616C61726D5FBD
:109A1800696E5F70726F6772657373203D3D206D6C
:109A2800616B655F7075626C69635F6964286964FE
:109A38005F686967682C206E6578745F69642900BF
:109A480064656661756C745F616C61726D5F706F7F
:109A58006F6C5F696E697469616C697A65642829DD
:109A680000000000616C61726D5F696420213D2017
:109A7800706F6F6C2D3E616C61726D5F696E5F70A7
:109A8800726F677265737300726300004174746566
:109A98006D7074656420746F20736C6565702069DF
:109AA8006E73696465206F6620616E2065786365F2
:109AB8007074696F6E2068616E646C65723B2075A6
:109AC800736520627573795F7761697420696620B0
:109AD800796F75206D75737400000000616C617298
:109AE8006D5F706F6F6C5F63616E63656C5F616CF7
:109AF80061726D00616C61726D5F706F6F6C5F6732
:109B080065745F64656661756C7400006765745F91
:109B1800656E7472795F69645F68696768000000E0
:109B280070685F667265655F6E6F6465000000004F
:109B380070685F6164645F6368696C645F6E6F64BA
:109B48006500000070685F696E736572745F6E6FA0
:109B58006465000070685F6765745F6E6F646500B8
:109B68006164645F616C61726D5F756E6465725F7C
:109B78006C6F636B000000007570646174655F75DD
:109B8800735F73696E63655F626F6F7400000000D6
:109B9800616C61726D5F706F6F6C5F616C61726D2B
:109BA8005F63616C6C6261636B0000006765745F82
:109BB800656E74727900000048617264776172653D
:109BC80020616C61726D20256420616C726561642E
:109BD8007920636C61696D656400000074696D6566
:109BE800725F68772D3E696E747320262031752068
:109BF8003C3C20616C61726D5F6E756D0000000009
:109C08002F55736572732F72712F7069636F2F7080
:109C180069636F2D73646B2F7372632F7270325F79
:109C2800636F6D6D6F6E2F68617264776172655FC7
:109C380074696D65722F74696D65722E630000001A
:109C480068617264776172655F616C61726D5F7380
:109C580065745F746172676574000000726F6F7479
:109C68005F6964002F55736572732F72712F706965
:109C7800636F2F7069636F2D73646B2F7372632F1B
:109C8800636F6D6D6F6E2F7069636F5F7574696C4C
:109C98002F70686561702E63000000002170685F96
:109CA8006765745F6E6F646528686561702C2072E3
:109CB8006F6F745F6964292D3E7369626C696E67A2
:109CC800000000002170685F6765745F6E6F6465EF
:109CD80028686561702C20726F6F745F6964292D24
:109CE8003E706172656E74006E65775F7375625F52
:109CF8007472656520213D20686561702D3E726F24
:109D08006F745F696400000070685F72656D6F76DC
:109D1800655F616E645F667265655F6E6F6465003E
:109D280070685F72656D6F76655F616E795F686593
:109D38006164000070685F6164645F6368696C6493
:109D48005F6E6F646500000070685F6765745F6EC2
:109D58006F64650076636F5F66726571203E3D20B3
:109D6800285049434F5F504C4C5F56434F5F4D4915
:109D78004E5F465245515F4B485A202A204B485A5D
:109D8800292026262076636F5F66726571203C3D28
:109D980020285049434F5F504C4C5F56434F5F4D0E
:109DA80041585F465245515F4B485A202A204B483C
:109DB8005A2900002F55736572732F72712F7069BD
:109DC800636F2F7069636F2D73646B2F7372632FCA
:109DD8007270325F636F6D6D6F6E2F68617264773A
:109DE8006172655F706C6C2F706C6C2E6300000084
:109DF8006662646976203E3D20313620262620663C
:109E080062646976203C3D203332300028706F73DD
:109E1800745F64697631203E3D203120262620700B
:109E28006F73745F64697631203C3D2037292026A2
:109E3800262028706F73745F64697632203E3D2057
:109E48003120262620706F73745F64697632203C57
:109E58003D203729000000007265665F66726571F3
:109E6800203C3D202876636F5F66726571202F2045
:109E780031362900706C6C5F696E697400000000EF
:109E880068616E646C6572203D3D20637572726511
:109E98006E74207C7C20657863657074696F6E5F72
:109EA80069735F636F6D70696C655F74696D655F19
:109EB80064656661756C742863757272656E742961
:109EC800000000002F55736572732F72712F70692F
:109ED800636F2F7069636F2D73646B2F7372632FB9
:109EE8007270325F636F6D6D6F6E2F686172647729
:109EF8006172655F657863657074696F6E2F6578E8
:109F080063657074696F6E2E630000006578636521
:109F18007074696F6E5F7365745F6578636C757371
:109F28006976655F68616E646C6572002C20667581
:109F38006E6374696F6E3A20000000006173736588
:109F48007274696F6E2022257322206661696C65C0
:109F5800643A2066696C6520222573222C206C697E
:109F68006E65202564257325730A000031203D3D68
:109F7800202875696E747074725F74296C2D3E7335
:109F880070696E5F6C6F636B000000002F5573651E
:109F980072732F72712F7069636F2F7069636F2DE1
:109FA80073646B2F7372632F7270325F636F6D6DA2
:109FB8006F6E2F7069636F5F72756E74696D652F50
:109FC80072756E74696D652E630000000A2A2A2A6C
:109FD8002050414E4943202A2A2A0A000A0000003C
:109FE8006E6F7420737570706F7274656400000012
:109FF80072756E74696D655F696E69740000000042
:10A00800666E692B00000000666E69006E616E0066
:10A01800666E692D000000008E310010A631001018
:10A02800A63100109A310010A6310010A631001098
:10A03800A6310010A6310010A6310010A63100107C
:10A04800A631001082310010A631001076310010C0
:10A05800A6310010A63100106A31001076320010C7
:10A068009C320010BA3200109C3200105632001098
:10A078009C3200109C3200109C3200109C32001060
:10A088009C3200109C3200109C320010923200105A
:10A098009C3200109C3200109C3200109C32001040
:10A0A8009C320010C632001034370010F63200100F
:10A0B800F6320010F6320010F6320010F6320010B8
:10A0C800F6320010F6320010F6320010F6320010A8
:10A0D800F6320010F6320010F6320010F632001098
:10A0E800F6320010F6320010F6320010F632001088
:10A0F800F6320010F6320010F6320010F632001078
:10A10800F6320010F6320010F6320010F632001067
:10A11800F6320010F6320010F6320010F632001057
:10A12800F6320010F63200106035001022350010AB
:10A1380060350010F6320010F6320010F6320010CA
:10A14800F6320010F6320010F6320010F632001027
:10A15800F6320010F6320010F6320010F632001017
:10A16800F6320010F6320010F6320010F632001007
:10A17800F63200100A330010F6320010F6320010E2
:10A18800F6320010F6320010F6320010F6320010E7
:10A19800F6320010F6320010F63200100A330010C2
:10A1A800AE3500100A33001060350010223500105B
:10A1B8006035001000000000000000000000F03FC3
:10A1C800000000000000244000000000000059408A
:10A1D8000000000000408F40000000000088C340DD
:10A1E80000000000006AF8400000000080842E4152
:10A1F80000000000D01263410000000084D797419E
:10A208000000000065CDCD416D697373696E6720EC
:10A21800646F75626C652066756E6374696F6E0035
:10A228002A282875696E74385F74202A29726F6D20
:10A238005F646174615F6C6F6F6B757028726F6DAE
:10A248005F7461626C655F636F6465282753272CB0
:10A258002027462729292D3229202A2034203E3D2F
:10A268002053465F5441424C455F56325F53495A2A
:10A27800450000002F55736572732F72712F706936
:10A28800636F2F7069636F2D73646B2F7372632F05
:10A298007270325F636F6D6D6F6E2F7069636F5F81
:10A2A800646F75626C652F646F75626C655F696E4B
:10A2B80069745F726F6D2E63000000005F5F6165F7
:10A2C8006162695F646F75626C655F696E6974006D
:10A2D8002A282875696E74385F74202A29726F6D70
:10A2E8005F7461626C652D3229202A2034203E3D3E
:10A2F8002053465F5441424C455F56325F53495A9A
:10A30800450000002F55736572732F72712F7069A5
:10A31800636F2F7069636F2D73646B2F7372632F74
:10A328007270325F636F6D6D6F6E2F7069636F5FF0
:10A33800666C6F61742F666C6F61745F696E6974A7
:10A348005F726F6D2E6300005F5F61656162695FB8
:10A35800666C6F61745F696E69740000446562754C
:10A3680067000000626F6F74325F77323571303882
:10A3780030000000312E352E310000007069636F07
:10A388005F77000072746F735F6361720000000092
:10A398004F6374203132203230323300060052507D
:10A3A800D3F0754264A3001006005250E182887F02
:10A3B8006CA3001006005250BBFF3CB684A30010EB
:10A3C8000D0A00007570646174655F75735F736969
:10A3D8006E63655F626F6F74000000005544001083
:10A3E8005944001065440010B54400109944001009
:10A3F800000000002F55736572732F72712F7069FA
:10A40800636F2F7069636F2D73646B2F7372632F83
:10A418007270325F636F6D6D6F6E2F7069636F5FFF
:10A42800737464696F5F7573622F737464696F5FA7
:10A438007573622E6300000055534220737464697B
:10A448006E202F207374646F7574000006005250DC
:10A4580053B4F4A140A40010737464696F5F7573FA
:10A46800625F696E697400007570646174655F7518
:10A47800735F73696E63655F626F6F7400000000DD
:10A488005261737062657272792050690000000031
:10A498005069636F00000000426F6172642043449A
:10A4A800430000005265736574000000000000005E
:10A4B80088A4001098A40010001C0220A0A400107A
:10A4C800ACA4001009025400030100807D080B00B1
:10A4D800020202000009040000010202000405242F
:10A4E80000200105240100010424020205240600BD
:10A4F800010705810308001009040100020A000091
:10A50800000705020240000007058202400000091A
:10A5180004020000FF00010512010002EF020140E1
:10A528008A2E0A000001010203010000282875692B
:10A538006E747074725F7420296E6578745F6275CA
:10A54800666665725F707472202620306231313120
:10A558003131317529203D3D203000002F5573657C
:10A5680072732F72712F7069636F2F7069636F2D0B
:10A5780073646B2F6C69622F74696E797573622FBF
:10A588007372632F706F727461626C652F7261737E
:10A5980070626572727970692F7270323034302F40
:10A5A8006463645F7270323034302E6300000000E0
:10A5B80068775F646174615F6F6666736574286E3F
:10A5C8006578745F6275666665725F70747229205B
:10A5D8003C3D205553425F445052414D5F4D4158D8
:10A5E80000000000556E68616E646C656420495215
:10A5F8005120307825780A007268706F7274203D97
:10A608003D2030006463645F656470745F786665DC
:10A61800720000006463645F656470745F6F7065E6
:10A628006E0000006463645F7365745F61646472E4
:10A63800657373006463645F696E745F656E6162FD
:10A648006C6500005F68775F656E64706F696E7433
:10A658005F616C6C6F6300006463645F696E69744A
:10A668000000000021286275665F6374726C202602
:10A67800205553425F4255465F4354524C5F4655FE
:10A688004C4C29002F55736572732F72712F7069A6
:10A69800636F2F7069636F2D73646B2F6C69622F02
:10A6A80074696E797573622F7372632F706F727429
:10A6B80061626C652F72617370626572727970691C
:10A6C8002F7270323034302F7270323034305F7500
:10A6D80073622E63000000006275665F6374726CBB
:10A6E8002026205553425F4255465F4354524C5FE3
:10A6F80046554C4C000000006570202564202573E9
:10A708002077617320616C7265616479206176617C
:10A71800696C61626C65000043616E277420636F29
:10A728006E74696E75652078666572206F6E206933
:10A738006E616374697665206570202564202573D1
:10A74800000000006F757400696E000073796E6315
:10A758005F65705F6275666665720000085100107B
:10A768006E500010A0500010D25000100851001078
:10A7780008510010EE500010A050001008510010B1
:10A78800085100100851001008510010085100101D
:10A798000851001008510010805000100856001091
:10A7A800E2550010AA570010BC550010AA57001017
:10A7B80030550010B2550010AA5700104C55001023
:10A7C80064550010FE570010F0570010365800105E
:10A7D800FE57001018590010385900104A58001038
:10A7E8009658001050590010555D0010115E001069
:10A7F800555E0010195F00104D6000100000000049
:10A8080028202820282073697A655F742029207001
:10A81800784E6577426C6F636B4C696E6B202920AC
:10A828002620282030783030303720292029203D34
:10A838003D2030002F55736572732F72712F706928
:10A84800636F2F4672656552544F532D4B65726E78
:10A85800656C5631302E362E312F706F72746162EE
:10A868006C652F4D656D4D616E672F686561705F12
:10A87800342E630028202820282073697A655F74A5
:10A88800202920707652657475726E202920262042
:10A89800282073697A655F74202920282030783051
:10A8A80030303720292029203D3D2030000000008D
:10A8B80028202820282070784C696E6B2D3E78421D
:10A8C8006C6F636B53697A6520292026202820281D
:10A8D80020282073697A655F742029203120292077
:10A8E8003C3C202820282073697A656F66282073ED
:10A8F800697A655F742029202A2028202820736916
:10A908007A655F742029203820292029202D2031BC
:10A9180020292029202920213D2030202920213DBF
:10A928002030000070784C696E6B2D3E70784E6553
:10A93800787446726565426C6F636B203D3D2028D4
:10A9480028766F6964202A293029000076506F72B2
:10A9580074467265650000007076506F72744D61C0
:10A968006C6C6F630000000070785969656C645303
:10A9780070696E4C6F636B203D3D202828766F69A7
:10A9880064202A29302900002F55736572732F72AD
:10A99800712F7069636F2F4672656552544F532D3E
:10A9A8004B65726E656C5631302E362E312F706FB6
:10A9B800727461626C652F54686972645061727454
:10A9C800792F4743432F5250323034302F706F72F3
:10A9D800742E63007578437269746963616C4E659F
:10A9E8007374696E6700000021287B2075696E7496
:10A9F80033325F7420756C495053523B205F5F615E
:10AA0800736D20766F6C6174696C652028226D7295
:10AA1800732025302C204950535222203A20223DC1
:10AA280072222028756C49505352293A3A293B2002
:10AA3800282875696E74385F7429756C49505352AB
:10AA4800293E303B7D29000070784C6F636B2D3EAA
:10AA58007370696E5F6C6F636B0000007570646182
:10AA680074655F75735F73696E63655F626F6F743A
:10AA78000000000078506F72744C6F636B496E74FD
:10AA880065726E616C5370696E556E6C6F636B574F
:10AA9800697468426573744566666F727457616954
:10AAA800744F7254696D656F7574000076506F72DB
:10AAB800744C6F636B496E7465726E616C53706928
:10AAC8006E556E6C6F636B57697468576169740073
:10AAD80076506F72744578697443726974696361FA
:10AAE8006C00000076506F72745969656C640000E0
:10AAF800784576656E7447726F7570002F5573656B
:10AB080072732F72712F7069636F2F467265655269
:10AB1800544F532D4B65726E656C5631302E362E60
:10AB2800312F6576656E745F67726F7570732E630B
:10AB3800000000002820757842697473546F5761CB
:10AB48006974466F7220262030786666303030305F
:10AB58003030554C2029203D3D2030007578426921
:10AB68007473546F57616974466F7220213D2030A9
:10AB7800000000002128202820785461736B476565
:10AB8800745363686564756C657253746174652881
:10AB980029203D3D20282028204261736554797082
:10ABA800655F742029203020292029202626202886
:10ABB80020785469636B73546F5761697420213D21
:10ABC80020302029202900002820757842697473D4
:10ABD800546F5365742026203078666630303030E4
:10ABE8003030554C2029203D3D2030007845766591
:10ABF8006E7447726F7570536574426974730000A0
:10AC0800784576656E7447726F75705761697442DE
:10AC18006974730070785175657565536574436F11
:10AC28006E7461696E6572002F55736572732F7249
:10AC3800712F7069636F2F4672656552544F532D9B
:10AC48004B65726E656C5631302E362E312F71750C
:10AC58006575652E630000007078517565756553DC
:10AC68006574436F6E7461696E65722D3E75784DBB
:10AC78006573736167657357616974696E67203CB2
:10AC88002070785175657565536574436F6E74618E
:10AC9800696E65722D3E75784C656E677468000044
:10ACA80028206354784C6F636B202920213D20288D
:10ACB800202820696E74385F7420292031323720AB
:10ACC80029000000707851756575650078526574C3
:10ACD80075726E20213D202820282028204261738B
:10ACE80065547970655F7420292030202920290057
:10ACF80070784E65775175657565000021282028A4
:10AD08002070764974656D546F5175657565203D81
:10AD18003D202828766F6964202A29302920292097
:10AD28002626202820707851756575652D3E757822
:10AD38004974656D53697A6520213D202820554264
:10AD4800617365547970655F742029203055202916
:10AD580020290000212820282078436F7079506F1F
:10AD6800736974696F6E203D3D2028202820426158
:10AD78007365547970655F74202920322029202951
:10AD8800202626202820707851756575652D3E751A
:10AD9800784C656E67746820213D20312029202970
:10ADA80000000000707851756575652D3E7578490D
:10ADB80074656D53697A65203D3D203000000000C0
:10ADC8002128202820707851756575652D3E70639F
:10ADD80048656164203D3D202828766F6964202AF3
:10ADE80029302920292026262028207078517565A9
:10ADF80075652D3E752E7853656D6170686F726547
:10AE08002E784D75746578486F6C64657220213DA5
:10AE1800202828766F6964202A29302920292029AA
:10AE2800000000002820707851756575652029009C
:10AE380021282028202820707642756666657220B1
:10AE480029203D3D202828766F6964202A29302949
:10AE580020292026262028202820707851756575FD
:10AE68006520292D3E75784974656D53697A65208A
:10AE7800213D2028205542617365547970655F74BF
:10AE88002029203055202920290000007851756597
:10AE980075650000765175657565416464546F5237
:10AEA800656769737472790078517565756553655E
:10AEB8006D6170686F726554616B65007851756576
:10AEC800756552656365697665000000785175653A
:10AED800756547656E6572696353656E6446726F22
:10AEE8006D495352000000007072764E6F746966A7
:10AEF800795175657565536574436F6E7461696ED4
:10AF08006572000078517565756547656E6572698B
:10AF18006353656E64000000785175657565476513
:10AF28006E65726963437265617465007851756511
:10AF3800756547656E65726963526573657400006F
:10AF4800785461736B0000002F55736572732F720C
:10AF5800712F7069636F2F4672656552544F532D78
:10AF68004B65726E656C5631302E362E312F7461FA
:10AF7800736B732E6300000075785072696F726985
:10AF88007479203C203332007578536368656475A2
:10AF98006C657253757370656E646564203D3D2001
:10AFA80028205542617365547970655F74202920A3
:10AFB8003055000049444C45000000007852657443
:10AFC80075726E20213D2028202D31202900000097
:10AFD8002820282028202820707844656C6179650D
:10AFE800645461736B4C69737420292D3E75784ED7
:10AFF800756D6265724F664974656D73203D3D20BD
:10B0080028205542617365547970655F7420292042
:10B01800302029203F202820282042617365547958
:10B0280070655F74202920312029203A20282028A3
:10B038002042617365547970655F7420292030203F
:10B0480029202920290000007578536368656475F4
:10B058006C657253757370656E64656420213D205C
:10B0680028205542617365547970655F74202920E2
:10B07800305500007578546F705072696F7269743A
:10B088007900000070784576656E744C69737400B9
:10B098007078556E626C6F636B6564544342000050
:10B0A800707854696D654F75740000007078546944
:10B0B800636B73546F576169740000007078544370
:10B0C80042203D3D20707843757272656E7454431A
:10B0D8004200000070785443422D3E75784D7574D7
:10B0E8006578657348656C640000000070785443A7
:10B0F8004220213D20707843757272656E74544306
:10B1080042000000765461736B5072696F72697403
:10B1180079446973696E68657269744166746572A9
:10B1280054696D656F757400785461736B507269FA
:10B138006F72697479446973696E686572697400BD
:10B14800785461736B436865636B466F7254696DBD
:10B15800654F757400000000765461736B52656D1D
:10B168006F766546726F6D556E6F72646572656451
:10B178004576656E744C6973740000007854617389
:10B188006B52656D6F766546726F6D4576656E7448
:10B198004C69737400000000765461736B506C61E5
:10B1A80063654F6E4576656E744C6973745265734A
:10B1B8007472696374656400765461736B506C6172
:10B1C80063654F6E556E6F7264657265644576652A
:10B1D8006E744C6973740000765461736B506C61C3
:10B1E80063654F6E4576656E744C69737400000034
:10B1F800765461736B537769746368436F6E7465D3
:10B2080078740000785461736B496E6372656D657C
:10B218006E745469636B0000785461736B52657384
:10B22800756D65416C6C0000765461736B53746185
:10B2380072745363686564756C65720076546173E3
:10B248006B44656C61790000707276496E69746947
:10B25800616C6973654E65775461736B000000001B
:10B268002820707854696D65722D3E7854696D6533
:10B2780072506572696F64496E5469636B73203EDE
:10B2880020302029000000002F55736572732F723B
:10B29800712F7069636F2F4672656552544F532D35
:10B2A8004B65726E656C5631302E362E312F7469AF
:10B2B8006D6572732E630000948E0010D88E001096
:10B2C800D88E00101C8F0010288F0010568F001089
:10B2D800D88E0010D88E00101C8F0010288F0010F8
:10B2E800546D725100000000546D72205376630053
:10B2F8007852657475726E0070727650726F6365FD
:10B3080073735265636569766564436F6D6D616ECD
:10B31800647300007854696D657243726561746581
:0CB3280054696D65725461736B00000085
:10B33400A4A30010B0A3001088020010BCA3001046
:10B3440094020010A0020010AC02001054A40010DB
:10B35400094B1B78002B08D00CE09A00802149058A
:10B36400511808680549505001333F2BF5DD024B55
:10B3740001221A707047C0463F1D02204C11002064
:10B3840010B5014B984710BD4D11002000280AD07C
:10B3940003231B02054A12685340C0229200134043
:10B3A400034A136070470223F3E7C0460C80014050
:10B3B4000C900140F0B5D6464F464646C0B507004E
:10B3C4000E00150018239A461B88142290461088F4
:10B3D40028499847814653461B8842461088264987
:10B3E4009847040053461B884246108823499847CF
:10B3F40080464B46002B0CD0002C0AD0002808D0E5
:10B40400FFF7A6FFC847A0470020FFF7BFFF2A00A9
:10B414000FE01B4B1B4A1C48802100F085FC002BCD
:10B4240007D0002A05D0C0235B051B6E3370013A98
:10B4340001362B00134312D0C0235B059C6A0823FA
:10B444002340A407EBD5002DE9D0511B0D29E6D8E4
:10B454003878C02149050866013D0137DFE701203E
:10B46400FFF794FFC047FFF78BFFE0BCBA46B14635
:10B47400A846F0BD49460000455800004643000078
:10B48400E493001024940010F892001070B50400A6
:10B494000268EFF3108572B61368002BFCD0BFF37B
:10B4A4005F8F63685A1C0BD000290ED00B600020FC
:10B4B4002368BFF35F8F00221A6085F3108870BD84
:10B4C40000F022FC60600120F2E70020F0E70000B9
:10B4D400F0B583B0040017001E000368002B17D0DA
:10B4E40000F012FC01902568EFF3108172B6286811
:10B4F4000028FCD0BFF35F8F656801350ED03A0099
:10B504003300200000F0F8FB0028ECD000200FE00E
:10B51400084B094A0948852100F006FC019B636039
:10B524002368BFF35F8F00221A6081F31088012023
:10B5340003B0F0BD1098001068980010D897001060
:10B54400F0B583B0070016001D0001A9FFF79EFFA8
:10B55400041E02D0200003B0F0BD00F0D5FB019B17
:10B564009842F7D032002B003800FFF7B1FF0400F7
:10B57400F0E710B582B00400684600F0ADFB009A15
:10B58400019B2000FFF7A4FF02B010BD10B50268B4
:10B59400EFF3108172B61368002BFCD0BFF35F8FFA
:10B5A4004368013305D001235B42436000F0B4FBE0
:10B5B40010BD034B034A0448B42100F0B5FBC04658
:10B5C400249800105C980010D897001010B5002340
:10B5D40008E00133DA00002108481150844662442F
:10B5E4005160DBB20E2BF4D90548F0229200002101
:10B5F40000F0AAFB034B044A1A6010BD000010506F
:10B60400401300200417002080011050F0B5CE46EE
:10B61400474680B585B0234B9F6D0024012603E087
:10B62400B74376000134E4B2002F36D01F2C34D84F
:10B634003E42F6D01C4B9E65630899460123634045
:10B6440001221A4090464B465D0045446D01174B5C
:10B65400ED18280000F02EFA0028E1D0134A4B46DA
:10B664005B0043445B01D3189A789146DB8A984681
:10B674000C22002101A800F067FB07236A465371DE
:10B684006B464A461A7243460393012101A800F00F
:10B6940039FA280000F09EF9C2E705B0C0BCB946EB
:10B6A400B046F0BD000011500030115000130020CE
:10B6B40070B584B0634A9823D55880239B022C002C
:10B6C4001C401D4240D0604B9A6A604B1A600024B3
:10B6D400002109E05E4B5B183C3300221A7000F035
:10B6E400ABF931000134E4B20F2C18D8A6013000B4
:10B6F4002030574BC0189B193B331B78022BF1D1D8
:10B70400534B9B193A331E78002EEBD0504BA101BA
:10B714005B183C331B78002BDCD13100E2E70029B5
:10B7240008D14C4B1B78002B04D14B4A9033802119
:10B734008902D150434B996C4905490D01220020DF
:10B7440000F00AFB8024A402EB0609D4EB0329D5FC
:10B7540080235B021C4301AB404A1A8000260BE0A5
:10B7640010231C43FFF752FFF0E701AB985D00F094
:10B77400A3FA0123C3700136012EF6D901AE0C22BF
:10B784000021300000F0E0FA06237370344A02AB63
:10B7940003CA03C30121300000F0B4F92E4B802208
:10B7A40092021A65EB0407D46B041ED42B042FD425
:10B7B400AC4241D104B070BD80235B011C43214BDA
:10B7C40000221A60FFF702FF01AE0C2200213000B4
:10B7D40000F0BAFA012373700121300000F092F9ED
:10B7E4001D4B802212031A65DEE78023DB011C4314
:10B7F40001AE0C220021300000F0A6FA042373707D
:10B804000121300000F07EF9134B10221A65CDE7B8
:10B8140080231B021C4301AE0C220021300000F0E7
:10B8240093FA052373700121300000F06BF90A4B81
:10B83400802212011A65BBE721006940094800F023
:10B844007BFAC0460000115000400540EC12002075
:10B85400001300203D1D0220003011500080FFFF26
:10B8640000001050ECA50010094B1B6C9B070CD476
:10B874008378DB09012B01D0002007E0C37E022B73
:10B8840001D0002002E0012000E000207047C04603
:10B894000000115010B5FFF7E7FF002809D0064B50
:10B8A4009B6A064A12689B1A054A94466344C62B4F
:10B8B40000D810BD0020FCE700400540EC12002039
:10B8C400E0FCFFFFF8B504000F00838A028B1E1C06
:10B8D400934200D9161CB6B29B1BA3828022D200CD
:10B8E4003243E378002B13D08025AD0115430122A8
:10B8F4005340E3706378002B0CD0A38A002B02D151
:10B904008023DB011D43002F00D02D042800F8BD47
:10B914000025EBE7E068BB01C0182169320000F0A4
:10B9240023FA23699B19236180231B021D43E4E747
:10B9340070B5040083681B68002900D01B0C9D05AA
:10B94400AD0D6278002A12D11B0409D4E38A5B1975
:10B95400E382238BAB4201D90023A382280070BD6C
:10B964000E4B0F4A81210F48490000F0DDF91B04FA
:10B974000DD52069E368890159182A0000F0F4F90B
:10B98400E38A5B19E38223695B192361E1E7064BD0
:10B99400034A0A210348FF3100F0C6F96CA60010DF
:10B9A40054A700108CA60010E0A6001010B50400E7
:10B9B40083681B680021FFF7BBFF63681B685B009B
:10B9C40002D5238B834200D010BD01212000FFF754
:10B9D400AFFFF9E7002383768382C3820361704754
:10B9E40010B5002902D083681B681940002A0FD0C3
:10B9F400114352050CD5826813685B050BD40B4BBD
:10BA04000B401360FFE7FFE7FFE7FFE7FFE7FFE710
:10BA14008368196010BD83787F211940DB09044ACB
:10BA24009B0004489A5800F087F9C046FFFBFFFFCB
:10BA3400980B002000A7001070B5040043681E682E
:10BA44000021FFF73FFF80256D010543164B1B6C5A
:10BA54009B0715D5A3785B0617D10023A28A002A79
:10BA640001D0002B15D0114B1E4080239B0533437E
:10BA7400626813602A0000212000FFF7B1FF70BD47
:10BA8400A378DB0903D10133E8E70123E6E70023C8
:10BA9400E4E701212000FFF715FF0543044A324083
:10BAA400A023DB051343E3E700001150FFFFFFAFC2
:10BAB400FFFFFFDF70B50400857E002D06D0FFF781
:10BAC40075FFA38A002B0BD1280070BD83787F21DA
:10BAD4001940DB09094A9B0009489A5800F02CF9DF
:10BAE4002000FFF7D7FE051E03D00123237700258E
:10BAF400EAE72000FFF7A0FFE6E7C046980B002026
:10BB040020A7001070B584B005004378042B48D0FA
:10BB140006D8022B23D0032B00D0A9E0002466E032
:10BB2400052B00D0A4E05C4B1B78DB0737D55A4AC1
:10BB3400137804218B431370584B1C682000143075
:10BB440000F0D2F82900200000F0BEF86269A36971
:10BB5400BFF35F8F0021116083F310881FE04E4B09
:10BB64001A7801218A431A701A7801318A431A70AB
:10BB740000265E701A7802318A431A70474B1C689B
:10BB84002000143000F0B0F82900200000F09CF8E8
:10BB94006269A369BFF35F8F166083F3108804B0F2
:10BBA40070BD3D4B1B78DB07F9D53B4A1378042164
:10BBB4000B431370394B1C682000143000F094F8C8
:10BBC4002900200000F080F86269A369BFF35F8F49
:10BBD4000021116083F31088E1E762001219D2009A
:10BBE4002F4B1B689B18002B13D10134E4B22D4B4F
:10BBF4001B78A34216D32C4A002A11D0A342ECD8B6
:10BC0400E31ADBB2002BF0D15A00D318DB00274A29
:10BC14009B185B69002BE8D0287869689847E4E7AB
:10BC24002300EFE71C4B1B785B07B8D51A4A13783F
:10BC340004218B4313700C22002101A800F084F826
:10BC44002B786A46137105235371144B1C6820002A
:10BC5400143000F049F801A9200000F035F86269B9
:10BC6400A369BFF35F8F0021116083F3108896E707
:10BC74000A4B1C682000143000F036F8290020001C
:10BC840000F022F86269A369BFF35F8F002111609D
:10BC940083F3108883E7C04620100020781000202A
:10BCA400F80C00203C1D022011450010F0A70010E4
:10BCB4007047C0460000000001B40248844601BC3D
:10BCC400604700BF694A001001B40248844601BCC1
:10BCD400604700BFCF68001001B40248844601BC2D
:10BCE400604700BF0F12001001B40248844601BC33
:10BCF400604700BFA54E001001B40248844601BC51
:10BD0400604700BF9D70001001B40248844601BC26
:10BD1400604700BF256F001001B40248844601BC8F
:10BD2400604700BF1570001001B40248844601BC8E
:10BD3400604700BF8524001001B40248844601BC5A
:10BD4400604700BFB525001001B40248844601BC19
:10BD5400604700BF1141001001B40248844601BC91
:10BD6400604700BF794B001001B40248844601BC0F
:10BD7400604700BF1D4100101000000000000000DB
:10BD840000000100000000000000000000000200AC
:10BD9400000000000000000000000300000000009C
:10BDA400000000000000FF000000000001B548682A
:10BDB40001318E460047704609380149884701BD64
:10BDC4003D1000104C0B002000000000F00B002080
:10BDD40080120020000000000000000090120020EB
:10BDE400000000000000000010000000000000003F
:10BDF400503300004C330000543300005233000031
:10BE04004D5300004D430000533400004334000000
:10BE140015490010000000008D4800104545001031
:10BE240000000000000100004CA7001050A7001003
:10BE34007C10002010000C00000000000000000036
:10BE4400000000000000000000000000FFFF0000F0
:10BE54001F000000000000000000000000000000BF
:10BE640000000000014100109D370010293E001021
:10BE740079400010E502001009060010B1710010AD
:04000005100001E9FD
:00000001FF
